:100000000C9466000C9487000C9487000C94870075
:100010000C9487000C9487000C9487000C94870044
:100020000C9487000C9487000C9487000C94870034
:100030000C9487000C9487000C9487000C94870024
:100040000C9487000C9487000C9487000C94870014
:100050000C9487000C94E80C0C9487000C94870097
:100060000C9487000C94A5110C9487000C948700C5
:100070000C9487000C9487000C9487000C948700E4
:100080000C9487000C9487000C9487000C94BE0D90
:100090000C9478190C9487000C9487000C948700BA
:1000A0000C9487000C9487000C9487000C948700B4
:1000B0000C9487000C9487000C9487000C948700A4
:1000C0000C9487000C9487000C94870011241FBEA9
:1000D000CFEFD1E2DEBFCDBF00E00CBF14E0A0E067
:1000E000B2E0EEEAFBE800E00BBF02C007900D9221
:1000F000AE32B107D9F717E0AEE2B4E001C01D920D
:10010000A831B107E1F70E94B9030C94D5450C94CE
:100110000000109234048091340480933304809161
:10012000330480933204809132048093310410921E
:1001300035040895EEE6F0E080818260808383E0FC
:1001400084BD85BD8AEF87BD0895E1E7F0E0808139
:1001500081608083089580917100817008958091FD
:100160008B04982F9295969596959370282F221F21
:100170002227221F9227282F22952F709227282F7F
:100180002695269592279170880F892B80938B0452
:100190000895909381048093800485EB9BE3909372
:1001A00093048093920483E393E190939904809362
:1001B000980485E694ED90938F0480938E040895BF
:1001C0008091800490918104AC01440F452F441F1D
:1001D000550B5195482759276091920470919304CB
:1001E00070938104609380048091980490919904A5
:1001F000909393048093920420918E0430918F0405
:100200003093990420939804C9010024969587950A
:100210000794969587950794982F802D822793278A
:1002200084279527542F44275295550F507E8427B5
:10023000952790938F0480938E04660F771F6F5FCE
:100240007F4F869F9001879F300D969F300D112420
:10025000C9010895FC019081992351F08091C80053
:1002600085FFFCCF9093CE00319690819923B1F712
:1002700008951F93CF93DF93182F492FE0E1F7E202
:10028000C0E0D0E0812F942FBF010E948C459B01DC
:100290006115710589F5812F942FBF010E948C454E
:1002A000182F492FCF016AE070E00E948C45FB01B6
:1002B0002196C430D10531F73097A1F18091C80063
:1002C00085FFFCCF812F942FBF010E948C45605D7C
:1002D0006093CE00CF016AE070E00E948C459B01E4
:1002E00061157105F9F0812F942FBF010E948C4593
:1002F000182F492FF901E2CF8091C80085FFFCCF6C
:10030000822F805D8093CE00812F942FBF010E94A9
:100310008C45182F492FCF016AE070E00E948C4570
:10032000FB01CACFDF91CF911F910895982F9F7045
:100330009A3040F48091C80085FFFCCF905D909387
:10034000CE0008958091C80085FFFCCF995C909302
:10035000CE000895CF93DF93EC01892F99278295E2
:100360008F700097C1F48D2F9927009789F4CE01E3
:10037000929582958F7089279F708927009711F039
:100380000E9496018C2F0E949601DF91CF910895D3
:100390000E949601ECCF0E949601E5CF982F8091A4
:1003A000C80085FFFCCF9093CE0080E090E00895D8
:1003B0002091C800332727FD30952227330F221FB5
:1003C0003327C90108958091C80087FFFCCF809131
:1003D000CE0090E008959C018FEF8093850493E018
:1003E000283E390768F5809382048093830424367D
:1003F0003105D8F0C90164E670E00E948C45609335
:100400008204C9016AE070E00E948C45CB016AE079
:1004100070E00E948C4580938304C9016AE070E01B
:100420000E948C458093840408952A30310548F752
:10043000C9016AE070E00E948C45809384040895AD
:100440001092820410928304109284040895909173
:100450003604936090933604809337040895809116
:1004600036048360809336040895F999FECF92BDD7
:1004700081BDF89A30B5F999FECF019692BD81BD44
:10048000F89A20B5932F80E030E0282B392BC90152
:100490000895F999FECF92BD81BDF89A80B508956F
:1004A000F999FECF92BD81BD60BDF894FA9AF99A90
:1004B00078940895FF920F931F938C01F62E672F67
:1004C0000E945002C80101966F2D0E9450021F9198
:1004D0000F91FF9008958091C90088618093C900B1
:1004E00083E38093CC001092CD008091C80087FDFB
:1004F00032C08091C90080688093C9008091C1009A
:1005000088698093C1008FE18093C4001092C50078
:1005100090EC91B98CE382B987E384B995B99FEFE8
:1005200097B988EF8AB98BE08BB982E08DB99EB913
:1005300010BA91BB13BA94BB8DB581608DBD81E5B6
:100540008CBD08958091CE008AE00E94F60D8091C6
:10055000C80087FFCECF8091C80087FDF3CF809180
:10056000C80087FFF8CFEECFEF92FF920F931F9353
:10057000CF93DF93EC0181E0CD32D80750F5C8323C
:10058000D105B0F588E290E090937D0480937C04DF
:1005900090938A04809389040E94331924E234EFF3
:1005A00030938D0420938C0482E08093910080919D
:1005B0008C0490918D04909581959F4F90938D041C
:1005C00080938C04DF91CF911F910F91FF90EF905A
:1005D00008958CE291E090937D0480937C04909345
:1005E0008A04809389040E9433192DE830E2D8CF21
:1005F000D0937D04C0937C04D0938A04C093890473
:10060000CE010E9433199E0140E050E060E070E7A7
:1006100088E399E30E94B345B901CA01969587958D
:10062000779567959695879577956795969587952C
:100630007795679526E030E040E050E00E94B345B2
:1006400079018A01C801AA27BB279C01887F892BD1
:1006500009F45FC0C901807F892B99F0C901807EB0
:10066000892BF1F0C901807C892B49F1C901807087
:10067000892BA1F120703C7F232BE1F11092910096
:1006800096CFF4E016950795F794E794FA95D1F78D
:10069000F0928D04E0928C0486E08093910087CFE5
:1006A000E5E016950795F794E794EA95D1F7F0926F
:1006B0008D04E0928C0487E08093910078CF76E0FF
:1006C00016950795F794E7947A95D1F7F0928D04F3
:1006D000E0928C0483E08093910069CFBB27A12F27
:1006E000902F8F2D90938D0480938C0484E08093C1
:1006F00091005DCF5AE016950795F794E7945A95C7
:10070000D1F7F0928D04E0928C0485E08093910003
:100710004ECFA3E016950795F794E794AA95D1F7E5
:1007200097013ECF85E090E00E9435020E94B4021E
:1007300080918C0490918D0490937F0480937E042B
:1007400010922F04E1E7F0E0808181608083809146
:100750007C0490917D04909391048093900408957B
:1007600085E20E945915E1E7F0E080818E7F808369
:100770000895AF92BF92CF92DF92EF92FF920F93C4
:100780001F93DF93CF93CDB7DEB760970FB6F89482
:10079000DEBF0FBECDBF0E946B020E94920380910C
:1007A0006E00826080936E0083E084BD85BD8AEF19
:1007B00087BD8BE696E09093AE068093AD06F999DF
:1007C000FECF82E090E092BD81BDF89A80B5982F6F
:1007D000937090932E048295817080936A04F999A6
:1007E000FECF87E090E092BD81BDF89A80B5882366
:1007F00011F0813208F080E180930002F999FECF78
:1008000083E090E092BD81BDF89A80B58F708093AF
:10081000AD04F999FECF84E090E092BD81BDF89AD5
:1008200080B58F7080939A0488E090E00E94350232
:1008300080938B0420917C0430917D04280F391F14
:10084000309381042093800485EB9BE39093930481
:100850008093920483E393E19093990480939804A6
:1008600085E694ED90938F0480938E040E94E000BF
:100870000E94E0000E94E000BC0188E090E00E943D
:100880005A02F999FECF8AE090E092BD81BDF89AB4
:1008900090B5892F8F708093940480919404833055
:1008A00010F01092940492959F709F5F909397041C
:1008B00080919704823008F4E2C00E94B32C7894AF
:1008C00000E010E01DC08091DA040E94F3150E9440
:1008D0002517C801849668E270E00E94A0450E9436
:1008E000BB180E94591580E10E94F60DC80187705F
:1008F0009070892B69F00F5F1F4F0C32110579F052
:10090000083208F7802F0E94BB180E942115DBCF08
:100910000E9474140F5F1F4F0C32110589F70E945B
:10092000D0150E9425170E94741480E00E94AF1217
:10093000882331F083E00E94AF12882309F0EBC0D6
:1009400083E00E94AF12882309F09DC08091DA04F1
:100950008093C40610920507109298051092210604
:1009600081E080932706109228068091C40660914A
:10097000050740912106209127060BE616E00E940C
:10098000B92B60912106C8010E94EA280E947528AF
:100990000E94741480913604836080933604109210
:1009A00037048091D504873009F466C0883030F56B
:1009B000823009F449C08330A8F5882309F44AC07D
:1009C000813009F444C00E9474140E947528882361
:1009D000F9F68091D5048630B1F781E00E94DB12F0
:1009E000882389F380E00E94AF12882361F30E947C
:1009F000D0150E942517E0E0F0EF19948C30C9F172
:100A00008D3038F4883061F18B30E9F60E9408228D
:100A1000BFCF8E3011F18E30A0F08F30A1F60E9442
:100A2000C92CB6CF843051F0843028F0853059F687
:100A30000E94BB31ADCF0E949724AACF0E94AC1C6C
:100A4000A7CF0E945044A4CF0E94D03BA1CF0E94C8
:100A5000EB3D9ECF0E943E119BCF0E940E1998CF76
:100A60000E94D0150E9474140E9475288823D1F327
:100A70008FCF0E94BC0F8CCF0E944E2689CF82E080
:100A8000809397041ACF8CE00E94AF12882309F458
:100A90005DCF7E010894E11CF11CBB2491E1C92EBD
:100AA000D12CCC0EDD1E8FE0A82E87010E94E00025
:100AB000F801908381830E5F1F4F0C151D05B1F760
:100AC000F70104C031960E171F0791F02081822F85
:100AD00090E08F7090700D9724F0822F8F7080833C
:100AE000282F2D3079F78E2F8E198F3009F072C094
:100AF00080E060E04B2D21E087010E942E2C85E5EF
:100B00000E94DA180E942517B394F0E8BF1669F620
:100B10000E94D0151BCF10922E0410926A0460918F
:100B20006A0470E06170707062957295707F7627CC
:100B3000607F762782E090E00E9450020E94B32CF2
:100B40001092AD0410929A0483E090E060E00E945D
:100B5000500284E090E060919A040E94500288E77D
:100B600090E090937D0480937C0485E090E068E7BA
:100B700070E00E945A0280E18093000260910002BE
:100B800087E090E00E9450021092940488E08093E5
:100B90009704809197046091940490E00197829566
:100BA0009295907F9827807F9827682B8AE090E025
:100BB0000E94500210E082E20E948D1583E20E94A2
:100BC0008D150E94251782E30E94F60D1F5F1832D3
:100BD00091F79ECFA08276CFCF92DF92EF92FF92D5
:100BE0000F931F93CF93DF93F89480912E0481305D
:100BF00009F4C1C280917304813009F4EDC1809180
:100C00003104863060F010923104809132048F5F9D
:100C100080933204809133048F5F809333048091FA
:100C20003304882341F08091330490E08370907006
:100C3000892B09F4BAC180913404883038F01092BD
:100C4000340480912E04882309F493C180913304E5
:100C50008F70809333049091320480910002981732
:100C6000C0F010923204809135048F5F8093350478
:100C70009091350480919704981708F077C180917E
:100C8000360482608093360480913A0481608093B8
:100C90003A0480911207882329F480913204882332
:100CA00009F45AC180913204882329F48091730495
:100CB000823009F447C28091D5048C3009F47BC19D
:100CC00080912E04882301F5909143048091E903DB
:100CD000981710F0109243048091430480FF2DC2B6
:100CE0005C988091430480FF0FC0809143048F5F24
:100CF000809343047894DF91CF911F910F91FF90DF
:100D0000EF90DF90CF900895809174042091E903D3
:100D10004091E90390E030E0240F311D82179307E2
:100D200014F010927404809174046091E903669544
:100D30000E948045992309F48AC0DD248091D5045E
:100D4000873009F490C0883008F063C1813008F022
:100D500007C280917304823009F433C28091120774
:100D6000882321F082E0D81609F436C28091120758
:100D7000882309F4FCC1809160048F708093600423
:100D80008091330490E08370907002970CF4AFC1AF
:100D900085E20E9459158091600490E08370907004
:100DA00002970CF4A1C18FEF8093580480916904DD
:100DB000882309F069C180917204882329F0809109
:100DC0003704882309F097C180913804882309F0FB
:100DD00049C10E942517DD2031F080912F048F5FDB
:100DE000817080932F042091890430918A0480912E
:100DF0007C0490917D042817390719F0C9010E94DD
:100E0000B402809174048F5F80937404809106070C
:100E10008F5F80930607809131048F5F8093310448
:100E2000809143048F5F8093430420910607809153
:100E3000E90330E0869586954CE0849FC00111243B
:100E40002817390714F010920607789454CF809130
:100E50002F04882309F469C1DD24D3948091D5043B
:100E6000873009F070CF81E0D81609F497C2E2E02C
:100E7000DE1609F06ECF809160048F5F809360046E
:100E800080911207882309F461C080919905882315
:100E900009F51092060780919D05882349F48091F9
:100EA0000807882329F080916904882309F03FC549
:100EB0008091210660916906680F8091AD0690913E
:100EC000AE060E94EA281092600480916404882390
:100ED00009F47AC480919905E091AD06F091AE06CF
:100EE000E80FF11D808180937B04809188048093BA
:100EF000860480917B0480748093880480916904C7
:100F0000882309F0DFC380917B048F708F3009F450
:100F10004FC480917B048F708F3071F080917B047F
:100F20000E940E299091B3066091860440917B0443
:100F30004078890F0E948D1C8091D504833009F47C
:100F4000EEC38091D504873009F4CBC38091360479
:100F5000816080933604FDCE80917304823009F065
:100F6000A1CE109273040E94D02F9CCE1092350413
:100F700086CE20917C0430917D04809190049091E4
:100F800091042817390709F461CE85E20E942115E2
:100F900060917C0470917D0470939104609390043F
:100FA00085E090E00E945A0251CE809134048F5F18
:100FB0008093340440CE80913A0480FF0AC080912F
:100FC0001207882309F090C180913F04882309F01B
:100FD000ECC210923A0474CE80911207882309F073
:100FE000A7C00E94D02F80912E04882309F0A2C0B0
:100FF000109234048091340480933304809133043C
:10100000809332048091320480933104109235042D
:1010100091C08B3009F427CF8C3008F0E1C08830C4
:1010200009F097CEF1E0DF1609F41AC382E0D81672
:1010300009F08FCE80917A048093300480917904F6
:1010400080937A040E94AF008093790480917A049F
:101050008F7360E040E00E948D1C80917A040E94B2
:10106000B50E77CE0E94CC188091330480FDB1CEAE
:10107000E0913304E695F0E0E370F070EE57FB4F3B
:1010800080810E94C118A5CE8CE20E940E29982F63
:10109000809160048111945F80910607882341F458
:1010A00080916A04882309F4D5C283E20E94211545
:1010B00080910607823009F07ECE80916A048823F1
:1010C00079F480916704823008F4E7C280912506A4
:1010D0000E940E2940912506407860E00E948D1CF8
:1010E00083E20E94591567CE109258045FCE85E2C4
:1010F0000E94211550CE80919404813009F43EC1A4
:1011000080919404882309F05FCE8091360480FF9B
:101110005BCE809136048E7F809336040E94E51565
:10112000809199050E94F3154FCEB2E0DB2E06CEDA
:101130000E946D2F1092730462CD5C9A88EF0E941A
:101140001C0FCFCD8091D504853009F4B4CD109219
:10115000740410922F041092990510927304ABCD71
:10116000843008F480CE853009F0F3CD7CCE81E266
:101170000E94591500CE0E9440128823A9F0809148
:101180007204882309F076C21092340480913404EA
:10119000809333048091330480933204809132042D
:1011A00080933104109235040E945212882309F46E
:1011B00021CD80917204882309F41CCD0E946D2FEB
:1011C00019CD81E20E9459158091310463E00E949B
:1011D0008045992309F0CFCD81E20E942115CBCD26
:1011E0008C3021F08D3009F0B4CD3DCE0E94E51554
:1011F00080913A0480FDD5C180913F04882309F095
:10120000CAC1E1E0DE1609F459C1F2E0DF1609F0C7
:10121000A0CD809160048F5F80936004809112075D
:10122000882309F496CDE0916906F0E0E155F94F85
:10123000808184FD3DC286E08093E9038091990519
:10124000E091AD06F091AE06E80FF11D808180932C
:101250007B04809188048093860480917B04807451
:101260008093880480917B048F708F3009F422C2B0
:1012700080917B048F708F3071F080917B040E948D
:101280000E299091B3066091860440917B044078CA
:10129000890F0E948D1C80913904982F92959F7020
:1012A0009093C406982F9770909321068695869503
:1012B000869581708093050780910507882309F042
:1012C000F0C188E00E94211581E00E9459150E941A
:1012D000CE16809121068F5F0E946E1680911207B4
:1012E00081708093120735CD80911207823008F407
:1012F00070CE80913F04882329F48091850588234E
:1013000009F467CE80914004809339049091690676
:101310009F5F90936906909169069170909369061A
:101320006091690670E062957295707F7627607FA4
:1013300076276559794F7093AE066093AD0690910C
:101340006906C92FD0E00E945C2BC155D94F888314
:10135000E0916906F0E0E155F94F80818F708F5F71
:101360008093EB03E0916906F0E0E155F94F80814D
:1013700084FD7EC186E08093E9032BCE8091360404
:1013800081FFBECE809136048D7F809336040E940B
:10139000E515809135040E94F315B2CE80919D052C
:1013A0008F5F80939D0580911207882309F4D1CC2B
:1013B000809199058F5F809399059091990580910F
:1013C000EB03981710F010929905809199058823E6
:1013D00009F06EC08091D504833009F420C110E07B
:1013E0008091D504873009F4A7C181E00E94B92813
:1013F000809169068F5F80936906C090690690911D
:10140000690680912706981708F443C08091640408
:10141000882319F481E0809371048091D504813090
:1014200009F4E5C18091D504823009F4DCC182E081
:101430000E94B92810929D0580916904882369F063
:10144000809167048093080780910807882329F01A
:101450001092670481E0809397051092690680914D
:10146000D504833009F400C28091D504873009F493
:10147000D5C180912806882309F0BCC19091050749
:1014800080919805981729F080916404823008F4BF
:1014900082C28091690690E082959295907F98270C
:1014A000807F98278559994F9093AE068093AD061B
:1014B00080916904882309F04CCC57C080911207B1
:1014C000882309F446CC809199058F5F8093990514
:1014D00080913F04882309F4D0C09091400480910A
:1014E00039048917D1F1F0906906F394FE220F2D8B
:1014F00010E0E801C295D295D07FDC27C07FDC27C1
:10150000C559D94F80914004BE010E945C2B015502
:10151000194FF8018083E0916906F0E0E155F94F39
:101520002081F801808190E030E08227932784FDBC
:1015300014C08091400480933904F0926906E091D0
:101540006906F0E0E155F94F80818F708F5F8093DD
:10155000EB03D093AE06C093AD06809199056091E0
:10156000EB030E9480459093990580919905E09145
:10157000AD06F091AE06E80FF11D808180937B04EB
:1015800080917B048F708F3009F47FC08091880434
:101590000E94A41CDECB80913F0481500E94F31571
:1015A00030CE8FE00E94F31527CE809140048093C7
:1015B00039040E94D02F80912E04882381F4109248
:1015C00034048091340480933304809133048093F5
:1015D000320480913204809331041092350480915A
:1015E00069068F5F80936906809169068170809398
:1015F00069066091690670E062957295707F762742
:10160000607F76276559794F7093AE066093AD067B
:1016100080916906C82FD0E08091390494CE8091E2
:1016200081059091820501969093820580938105B2
:10163000209181053091820580918C0590918D05D6
:101640002817390708F4CBCE109282051092810535
:1016500011E0C6CE892F60E040E00E948D1C25CDB0
:1016600080E00E94A41C80917A040E94F40E71CB49
:1016700088E081CE0E94D02F87CD80918505882378
:1016800009F06BCF0E946D2F68CF8091880488236A
:1016900009F096C01092880479CF80E00E94A41CC3
:1016A0001FCD88E00E94591581E00E9421150FCEC0
:1016B00088E0C2CD80917B048F7080937B04109270
:1016C0008804D6CD809121066091270640919A0525
:1016D0002091280600919E05E09098050E9414181C
:1016E0002BCC80913804813009F419C18091810597
:1016F00090918205E0919205F0E0EE0FFF1FEF5F01
:10170000FD4F6081718182959295907F9827807FAF
:1017100098270E948C45862F0E94FE1517CC809139
:101720003804813009F00DCC8091810590918205BB
:1017300001960E94EB0105CC80915F04813009F095
:1017400054CE609105078091210640916906209151
:10175000B306480F89E895E00E940C1E809192051F
:101760006091810570918205409189050E94721EE9
:1017700080918105909182050196909382058093D6
:101780008105E09192052091810530918205F0E07C
:10179000EE0FFF1FEF5FFD4F808191812817390702
:1017A00008F423CE10925F0483E20E9459151DCEE7
:1017B00080917B048F7080937B0410928804A9CB66
:1017C00081E00E94A41C66CF8091210660912706CB
:1017D00040919A052091280600919E05E090980579
:1017E0000E94141877CB81E08093710420CE8093FF
:1017F000710418CE0E94A62880916404823008F0FB
:1018000048CE8091C4066091050740912106209141
:1018100027060BE616E00E94B92B3BCE80915F04B1
:10182000813009F026CE80918505882309F0B8C063
:1018300080918605882309F41CCE1092860580913C
:10184000920560918105709182056C190E94391E84
:10185000809192050E94CC1E9093940580939305ED
:1018600080E00E94591505CE80918505882309F0F6
:1018700079C080918605882309F44EC010928205B4
:10188000109281058091D0048093920580919205F9
:101890000E94D51E90938D0580938C0580919205B2
:1018A0000E94CC1E909394058093930520919305FC
:1018B0003091940580918C0590918D0528173907FA
:1018C00020F010929405109293058091860588234C
:1018D00009F053C080919205609181057091820555
:1018E0000E94261F80938905809192056091890549
:1018F00040EE55E028E935E00AE915E0ECEAEE2E85
:10190000E6E0FE2E0E94EC1D81E080932806809187
:10191000AC068093B306A8CD1123B9F2AFCF809166
:1019200081059091820501960E94EB01DFCE81E056
:101930000E94A41C80E00E94A41C609127068BE6F4
:1019400096E045EC56E02FE935E00E94192A109206
:1019500069048AE00E942A291092880482E00E9489
:10196000F60DA6CA10928505109282051092810587
:1019700083E20E94591511E07CCF10928605809178
:10198000930590919405909382058093810580E062
:101990000E9459159FCF809198058093050731CFFC
:1019A00010925F04109285058091920560918105E7
:1019B000709182050E94491E809192050E94D51E59
:1019C00090938D0580938C0583E20E94591530CF4A
:1019D0001F920F920FB60F920BB60F9211241F9306
:1019E0002F933F934F935F936F937F938F939F9327
:1019F000AF93BF93EF93FF9320B1227090B180918A
:101A000096042817F1F0892F8170222309F47AC0F7
:101A1000882309F47AC08091890490918A040197FF
:101A200090938A048093890431E08D32930708F4FF
:101A30007AC08CE291E090938A0480938904209389
:101A4000960480914C048F3F29F080914C048F5F65
:101A500080934C0480914D048F3F29F080914D0478
:101A60008F5F80934D0480917704909178048F5F0D
:101A70009F4F49F08091770490917804019690935C
:101A800078048093770480915B0490915C048F5F6D
:101A90009F4F49F080915B0490915C040196909374
:101AA0005C0480935B0410912E04113009F445C04E
:101AB0008091460490914704892B81F080914604DF
:101AC0009091470401979093470480934604809136
:101AD000460490914704892B09F45C98FF91EF919B
:101AE000BF91AF919F918F917F916F915F914F9136
:101AF0003F912F911F910F900BBE0F900FBE0F9033
:101B00001F901895882309F486CF809189049091BD
:101B10008A04019690938A048093890431E08D327F
:101B2000930708F086CF889708F089CF88E290E085
:101B300090938A048093890482CF99B19295917091
:101B400080914A04882319F090934A04C7CF9923BF
:101B5000D9F38091440490914504019690934504F3
:101B60008093440410924504109244040E94EC05B2
:101B700088EF0E941C0F10934A04B0CF1F920F925F
:101B80000FB60F920BB60F9211242F933F934F93E2
:101B90005F936F937F938F939F93AF93BF93EF93D5
:101BA000FF9380917E0490917F04909395008093A1
:101BB000940080918C0490918D0490937F04809385
:101BC0007E040E94EC05FF91EF91BF91AF919F9130
:101BD0008F917F916F915F914F913F912F910F90D6
:101BE0000BBE0F900FBE0F901F90189520EA3FE09C
:101BF000E22FF32F3197F1F78A95D1F708958823D3
:101C000009F41EC09AEF20EA3FE0E22FF32F31974C
:101C1000F1F79A95D1F7E22FF32F3197F1F79A95D3
:101C2000D1F7E22FF32F3197F1F79A95D1F7E22F01
:101C3000F32F3197F1F79A95D1F7815009F0E5CF5D
:101C400008951092A3041092AC0408951F93CF93AB
:101C5000DF93EC01142F6F777885772309F44CC05C
:101C6000462F50E0888190E08F7790704817590791
:101C700079F121E030E00DC0D901FE01E20FF31F40
:101C8000808190E08F7790702F5F3F4F841795078A
:101C900009F1271788F3272F2F5F293030F128E02B
:101CA000922F822F9150FE01E80FF11DDE01A90F46
:101CB000B11D8C918083892F9923A1F71536C0F42B
:101CC00080E0862B88832887DF91CF911F9108952C
:101CD000A0E0B0E0153670F480E0AC0FBD1F862B9D
:101CE0008C93DF91CF911F9108952223C9F6E6CFFF
:101CF00080E8E7CF80E8F1CF91E081E021E0D2CF2A
:101D0000CF93DF93EC0138853323B9F06F7770E020
:101D1000888190E08F7790706817790789F0FE01CD
:101D200020E008C0818190E08F779070319668172D
:101D3000790739F02F5F2317A8F3DF91CF9108952A
:101D400020E0323068F0922F9F5FFE01E20FF11D1C
:101D5000DE01A90FB11D8C918083292F9317A0F369
:101D600031503887DF91CF910895282F90919A04B0
:101D70008091C00085FFFCCF90699093C600822FB0
:101D800090E08F739070892BB1F48091C00085FF33
:101D9000FCCF1092C600822F82958695869583701F
:101DA00080FD19C0909123028091C00085FFFCCF77
:101DB0009093C60008958091C00085FFFCCF822FCC
:101DC0008F73875E8093C600822F82958695869555
:101DD000837080FFE7CF909121028091C00085FF42
:101DE000FCCF9093C6000895282F90919A0480917B
:101DF000C00085FFFCCF90689093C600822F90E0D2
:101E00008F739070892B39F48091C00085FFFCCFCF
:101E10001092C60008C08091C00085FFFCCF2F73D0
:101E2000275E2093C600909122028091C00085FF1A
:101E3000FCCF9093C6000895982F8091C00085FF35
:101E4000FCCF9093C60080E090E00895909141040B
:101E50008091420420E030E0981711F021E030E05A
:101E6000C901089590914104809142049817D1F3DB
:101E7000F89490914104E92FF0E0E255FB4F808106
:101E80009F5F90934104909141049F71909341040E
:101E9000789490E0089590914104809142049817BD
:101EA00029F00E94320F482F87FD03C040E0842FA5
:101EB0000895582F52955F705F30C9F3282F30E096
:101EC0002F7030708091AD0490E02817390771F7BA
:101ED00050933C04ECCF90919A048091C00085FF10
:101EE000FCCF906B9093C6008091C00085FFFCCF23
:101EF0008BE78093C6008091C00085FFFCCF1092D5
:101F0000C600089580912E04823049F08091C0006F
:101F100085FFFCCF8CEF8093C6000E946B0F089565
:101F2000909130048913089580E00E94A41C8FEFE3
:101F30008093300408951F93182F962F6623B9F0CD
:101F400060E0809130048F3F09F061E0953648F4FD
:101F5000812F895140E00E948D1C109330041F9105
:101F60000895812F895141E00E948D1CF6CF60E0D9
:101F70000E94900F1F910895FF920F931F938091DD
:101F80008505817080938505809185058093720415
:101F90000E94D01580918505882309F02EC10E94EA
:101FA00025178BE090E00E944902809324028CE088
:101FB00090E00E94490280932502FF2410E00E94D5
:101FC00074140E947528882309F048C09091410438
:101FD00080914204981769F00E94320F682F87FDA4
:101FE0006BC080913C04883009F4ACC0893009F49E
:101FF00077C0112371F42091A304222349F4809126
:10200000AC04882329F480911207882309F4E0C0E6
:1020100010E087E10E940413882389F280918505EE
:102020008F5F8093850580918505817080938505FC
:10203000809185058093720480E00E9459158091FB
:102040008505882309F4BBCF80E00E9421150E94FA
:1020500074140E947528882309F4B8CF0E946B0F6E
:1020600081E0809327068091050780939805109260
:1020700028068091C40660910507409121062091B1
:1020800027060BE616E00E94B92B60912106C801D5
:102090000E94EA28FF2061F08BE090E0609124022A
:1020A0000E9450028CE090E0609125020E94500254
:1020B0001F910F91FF900895482F42954F704F3018
:1020C00009F498C0282F30E02F7030708091AD0453
:1020D00090E02817390709F48DC010923C046FCFA7
:1020E00067FDBAC0062F0E94320F482F112309F056
:1020F00090CF50912402051748F0852F90E00F965D
:10210000202F30E0821793070CF082C050912502F7
:10211000051708F470CF852F90E00C96202F30E043
:10212000821793070CF467CF051B84EA94E0602FB5
:102130000E94260E8091A4048F778093B30620918D
:10214000A3045BCF67FD84C0062F0E94320F1123CA
:1021500071F540912402041748F0842F90E00F9607
:10216000202F30E0821793070CF06BC040912502BE
:10217000041708F440CF842F90E00C96202F30E015
:10218000821793070CF437CF041B84EA94E0602F86
:102190000E94800E8091AC04882309F42CCF80919A
:1021A000A4048F778093B3062091A30426CF113027
:1021B00009F456C089E10E945915009325028091C7
:1021C0008505809372042091A304FF24F39415CF16
:1021D00084E00E9404138823A1F485E00E94041384
:1021E000882309F415CF1092720489E10E94211509
:1021F00012E00FCF40933C04F4CE80E00E94211502
:10220000CECE1092720480E20E94211511E001CF1F
:10221000051B8BE994E0602F0E94260E2091A304F9
:1022200020933F0480919B048F778093400480919A
:10223000DA04909140048295807F890F8093400456
:10224000DCCE041B8BE994E0602F0E94800EE6CF69
:102250000E94320F082F79CF0E94320F082F43CFF0
:1022600080E20E9459150093240280918505809395
:1022700072042091A304FF24F394BFCE1F930E9405
:10228000E5158091AD040E94F3150E94741484E654
:102290000E94F60D0E94741484E60E94F60D0E94BE
:1022A00074148FEF809330040E9474140E94752878
:1022B000882301F590914104809142049817A1F37D
:1022C0000E94320F482F87FD19C080913C0488304E
:1022D00039F1893049F747FD30C0142F0E94320F81
:1022E000682F812F0E949B0F0E9474140E947528F2
:1022F000882301F30E946B0F1F910895582F529568
:102300005F705F30B9F0282F30E02F70307080910F
:10231000AD0490E02817390769F010923C04C4CF4F
:1023200047FD0FC0142F0E94320F682F812F0E948B
:10233000900FBACF50933C04C8CF0E94320F182F91
:10234000CDCF0E94320F182FEECF1F920F920FB6F3
:102350000F920BB60F9211242F933F934F935F93DD
:102360006F937F938F939F93AF93BF93EF93FF935D
:102370009091C6009A3F09F442C09C3FA9F1983F52
:1023800009F44AC080914204E82FF0E0E255FB4F87
:1023900090838F5F80934204809142048F71809379
:1023A00042049091420480914104981751F4809125
:1023B00041048F5F80934104809141048F71809329
:1023C0004104FF91EF91BF91AF919F918F917F91C8
:1023D0006F915F914F913F912F910F900BBE0F9096
:1023E0000FBE0F901F90189580917204882349F3B7
:1023F00080912E04823029F70E946D2FE2CF8091C8
:102400002E048230F1F680917204882311F00E942C
:10241000D02F0E948900D5CF8091770490917804C5
:1024200090932D0480932C041092780410927704DA
:1024300080912E04823029F680913D0490913E04D3
:10244000019690933E0480933D045C9A8091C00075
:1024500085FFFCCF88EF8093C6000E94EC05809139
:102460002C0490912D049695879580934604A9CFCE
:102470005F9A089580912E04813009F05F98089545
:1024800099B1991F9927991F80914804882311F4C5
:10249000992321F49093480480E008959093480490
:1024A00081E0089599B1991F9927991F8091490456
:1024B000882311F0992321F09093490480E0089536
:1024C0001092490481E008958AB1806F8AB98BB176
:1024D0008F708BB908958AB18F708AB98BB18F7064
:1024E0008BB90895AC01F894289800000000000012
:1024F0000000289A20E030E01EBC0DB407FEFDCF9E
:102500008EB5FA01E20FF31F80832F5F3F4F233018
:10251000310591F77894089516980895169A0895BC
:1025200020B1269526952F70822F90E02695322F88
:10253000369536952270322B880F991F282F2470DC
:10254000322B880F991F880F991F8870382B8FE0C6
:10255000831B089580B1869586958F700895282FE6
:10256000883188F4E82FE695E695E695F0E0E552A7
:10257000FB4F808190E0277002C0959587952A9542
:10258000E2F78170089580E00895282F883188F45B
:10259000E82FE695E695E695F0E0EE52FB4F808158
:1025A00090E0277002C0959587952A95E2F7817093
:1025B000089580E00895282F883188F4E82FE69563
:1025C000E695E695F0E0EA52FB4F808190E02770B7
:1025D00002C0959587952A95E2F78170089580E06D
:1025E00008958091DB04882321F48091DC04882302
:1025F00019F090E0892F089590E08091DD04882300
:10260000C9F791E0892F0895282F8831A0F4482F29
:10261000469546954695277081E090E0382F01C099
:10262000330F2A95EAF7A42FB0E0FD01EE52FB4FDD
:102630008081832319F420E0822F0895232F30E036
:1026400020953095A552BB4F8C9190E028233923DB
:10265000232B89F7342F3F5F832F63E00E9480454F
:10266000E92FF0E0E552FB4F8081882321F720E03D
:10267000832F8F5F0E948045E92FF0E0E552FB4FEA
:1026800080818823C9F621E0D7CF1F93CF93DF93B2
:10269000C8E3D2E010E088810E94AF12882329F4B9
:1026A0001F5F21961D30B9F71FEF812FDF91CF916A
:1026B0001F9108951F93CF93DF93C8E3D2E010E0FA
:1026C00088810E94C512882349F41F5F21961D301E
:1026D000B9F780E0DF91CF911F910895812F8F5F2F
:1026E000DF91CF911F9108951F93CF93DF93C8E39C
:1026F000D2E010E088810E94DB12882349F41F5F3A
:1027000021961D30B9F780E0DF91CF911F91089598
:10271000812F8F5FDF91CF911F9108951F93CF93EA
:10272000DF93C0E3D2E010E088810E94AF128823DB
:1027300049F41F5F21961830B9F780E0DF91CF91FF
:102740001F910895812F8F5FDF91CF911F91089581
:102750001F93CF93DF93C0E3D2E010E088810E9403
:10276000C512882349F41F5F21961830B9F780E01D
:10277000DF91CF911F910895812F8F5FDF91CF91CE
:102780001F9108951F93CF93DF93C0E3D2E010E031
:1027900088810E94DB12882349F41F5F219618303C
:1027A000B9F780E0DF91CF911F910895812F8F5F5E
:1027B000DF91CF911F910895CF93DF93C0E3D2E0D3
:1027C00088810E94AF12882349F4219682E0C833A1
:1027D000D807B1F780E0DF91CF91089581E0DF91D4
:1027E000CF910895FF920F931F93CF93DF93C0E390
:1027F000D2E0FF2400E006C00F5F219682E0C833DC
:10280000D80789F01881812F0E94AF128823A1F781
:10281000812F0E94DB12882381F3F394219682E0BA
:10282000C833D80779F781E0F81639F080E0DF91F6
:10283000CF911F910F91FF90089580E00730B9F775
:1028400081E0F5CF1F93CF93DF93C6E2D2E010E093
:1028500088810E94C512882349F41F5F21961A308F
:10286000B9F780E0DF91CF911F910895812F8F5F9D
:10287000DF91CF911F91089580914B0410924B04EA
:10288000089580E00895382F883100F5282F2770AB
:1028900081E090E0982F01C0990F2A95EAF7832FE5
:1028A000869586958695A82FB0E0FD01EE52FB4FE8
:1028B0008081892369F4FD01EA52FB4F80818923DD
:1028C00071F4A552BB4F8C91982339F480E00895A0
:1028D000832F0E94F41782E0089583E00895832FE8
:1028E0000E94FC1781E00895EF92FF920F931F93CF
:1028F000DF93CF9300D000D0CDB7DEB71092D204D3
:102900001092D6041092D3041092D7041092D404DB
:102910001092D80480914C048A3068F426960FB641
:10292000F894DEBF0FBECDBFCF91DF911F910F9105
:10293000FF90EF90089510924C0416987E01089431
:10294000E11CF11CC7010E9472128091DB048C8390
:102950008091DC048D838091DD048E8360E070E0E3
:1029600001E010E0E62FE695E695E695F0E0CB0174
:1029700087709070980102C0220F331F8A95E2F78A
:10298000C901AF0145525B4FD701AE0FBF1F3C914C
:10299000E252FB4F2081232B28238095FA013081BE
:1029A0008323282B20836F5F7F4F68317105D1F619
:1029B0000E949012982F96959093DA048093D004F9
:1029C000169A40E050E0BE016C5F7F4FDA01A252E0
:1029D000BB4FF701E40FF51F80818C93FB01E40FDF
:1029E000F51F2081FA01E552FB4F9081FA01EE526A
:1029F000FB4F822F809589238083FA01EA52FB4F97
:102A00009095922390834F5F5F4F43305105F1F6CD
:102A100090B1969596959F708091CE04891721F07C
:102A200010924D049093CE0480914D048F3630F077
:102A30009093CF048091CF048093CE040E942517F9
:102A40006DCF282F8832C0F4E82FE695E695E695FD
:102A5000F0E0277081E090E001C0880F2A95EAF746
:102A6000DF01A25BBB4F2C91282B2C93ED5AFB4F1F
:102A700080952081822380830895282F8832C0F496
:102A8000E82FE695E695E695F0E0277081E090E086
:102A900001C0880F2A95EAF7DF01AD5ABB4F2C9190
:102AA000282B2C93E25BFB4F80952081822380832F
:102AB0000895282F8832C8F4E82FE695E695E69524
:102AC000F0E0277081E090E002C0880F991F2A95FE
:102AD000E2F78095DF01A25BBB4F2C9128232C935A
:102AE000ED5AFB4F2081822380830895282F88325E
:102AF00098F4E82FE695E695E695F0E0ED5AFB4F61
:102B0000277081E090E002C0880F991F2A95E2F7B4
:102B100080952081822380830895282F883290F425
:102B2000E82FE695E695E695F0E0E25BFB4F27702F
:102B300081E090E002C0880F991F2A95E2F720817A
:102B4000282720830895E82F883298F4282F2770AB
:102B500081E090E002C0880F991F2A95E2F7E69580
:102B6000E695E695F0E0ED5AFB4F20812823822F71
:102B7000089520E0822F0895982F96959695969522
:102B8000EEE4F4E0E90FF11D208130E0877002C02F
:102B9000359527958A95E2F721703070C90108951F
:102BA00010925204109251041092500410924F044B
:102BB00010924E041092570410925604109255042D
:102BC00010925404109253040895CF93DF93C4EAF3
:102BD000D2E089910E94591582E0C43BD807C9F719
:102BE000DF91CF910895803108F00895E82FF0E04B
:102BF000EC55FD4F80810E94211508950F931F937E
:102C0000CF93DF93082FC4EAD2E010E007C0888199
:102C10000E9421151F5F2196103149F01017B8F35B
:102C200088810E9459151F5F21961031B9F7DF91F5
:102C3000CF911F910F910895803108F00895E82FEA
:102C4000F0E0EC55FD4F80810E943D1508958031E4
:102C500010F080E00895E82FF0E0EC55FD4F808102
:102C60000E94BC150895803110F080E00895E82F8F
:102C7000F0E0EC55FD4F80810E94A3150895883146
:102C800008F00895E82FF0E0E158FD4F80810E94A0
:102C900021150895883108F00895E82FF0E0E158F3
:102CA000FD4F80810E943D150895883108F00895F8
:102CB000E82FF0E0E158FD4F80810E9459150895FA
:102CC000CF93DF93CFE7D2E089910E94591582E03C
:102CD000C739D807C9F7DF91CF910895E82F815000
:102CE000883008F00895F0E0EA58FD4F80810E9496
:102CF000211508950F931F93CF93DF93082FC7E7F4
:102D0000D2E011E007C088810E9459151F5F21960B
:102D1000193069F01017B9F7E12FF0E0EA58FD4FCC
:102D200080810E9421151F5F2196193099F7DF914C
:102D3000CF911F910F910895E82F8150883008F0AE
:102D40000895F0E0EA58FD4F80810E9459150895DA
:102D5000E82F8150883008F00895F0E0EA58FD4FE0
:102D600080810E943D150895E82F8150883010F031
:102D700080E00895F0E0EA58FD4F80810E94A3159D
:102D80000895E82F8150883010F080E00895F0E039
:102D9000EA58FD4F80810E94BC150895CF93DF93C0
:102DA000C7E7D2E089910E94591582E0CF37D80752
:102DB000C9F7DF91CF9108958D3008F00895E82F7D
:102DC000F0E0E956FD4F80810E94211508958D3075
:102DD00008F00895E82FF0E0E956FD4F80810E9449
:102DE000591508958D3008F00895E82FF0E0E95660
:102DF000FD4F80810E943D150895E7E9F2E0E80F5C
:102E0000F11D80810E94A3150895CF93DF93C7E938
:102E1000D2E089910E94591582E0C43AD807C9F7D7
:102E2000DF91CF9108950E94051784E00E94591503
:102E300083E00E94591588E00E94591581E00E94A4
:102E4000591582E00E9459150895F894179820E0CA
:102E500030E090915804F901ED5AFB4F808198239E
:102E6000F901E25BFB4F8081982B9EBD0DB407FEFC
:102E7000FDCF2F5F3F4F2530310559F7179A7894D2
:102E80000895EEE4F4E0A3E5B4E080819D91892B00
:102E9000819384E0E335F807C1F70895EEE4F4E0A8
:102EA000A3E5B4E09D91909580818923819384E08E
:102EB000E335F807B9F70895EEE4F4E0A3E5B4E0EC
:102EC00020819C91892F822319F0909592239083E1
:102ED0001D92319684E0E335F80791F708951F932A
:102EE000182F84E00E945915123049F083E00E94A7
:102EF0005915113071F01F3F39F01F91089583E08B
:102F00000E943D151F91089584E00E9421151F9194
:102F1000089583E00E9421151F9108950F931F9338
:102F2000CF93DF93182F87FD50C086E10E9455167E
:102F3000812F829586958695837080FF29C085E1D3
:102F40000E943F161F7349F11731A0F58FEF0E94C1
:102F50006F1784E10E945516012F10E0CBE0D0E0FE
:102F6000C017D10731F0FE01E457FD4F80810E9468
:102F700059152196C831D10599F704571D4FF8010D
:102F800080810E942115DF91CF911F910F910895AB
:102F900085E10E9455161F73B9F680E00E946F17F5
:102FA0000E94051784E10E943F16DF91CF911F9187
:102FB0000F910895143268F0103370F4185181E0C5
:102FC0000E946F17112329F6EBCF86E10E943F166E
:102FD000AFCF1C5080E0F4CF1C3318F4145282E0C1
:102FE000EFCF105383E0ECCFEFE7F2E0E80FF11DF5
:102FF00080810E9421150895EFE7F2E0E80FF11DAE
:1030000080810E9459150895E7E7F2E0E80FF11D6D
:1030100080810E9421150895E7E7F2E0E80FF11D95
:1030200080810E9459150895DF92EF92FF920F93CD
:103030001F93CF93DF93F02EDE2C222371F1022F0A
:10304000040FE42EC7E7D2E010E00BC0101758F4CD
:103050001F15D9F088810E9421151F5F2196183015
:1030600049F01E1598F788810E9459151F5F219617
:103070001830B9F781E08D15A0F4DF91CF911F9141
:103080000F91FF90EF90DF900895E12FF0E0E95865
:10309000FD4F80810E943D15E0CF062F080FE82EDE
:1030A000D1CFDD2071F088E00E94591581E00E94A7
:1030B0002115DF91CF911F910F91FF90EF90DF903D
:1030C000089588E00E94211581E00E945915DF9142
:1030D000CF911F910F91FF90EF90DF900895FF9295
:1030E0000F931F93082FF62E84E00E94591583E05A
:1030F0000E94591588E00E94591581E00E945915D7
:10310000102F04FD34C015FD29C007FD2CC016FD8D
:1031100021C00E940517FF2099F0802F8F708D30FD
:1031200098F08BE10E9421158CE10E9421158FE01F
:103130000E9421158EE00E9421158DE00E9421152C
:103140001F910F91FF9008950E94DC161F910F911F
:10315000FF90089581E00E942115DBCF83E00E945B
:10316000211507FFD4CF88E00E942115D0CF84E03D
:103170000E942115C8CFE5E4F2E0E80FF11D80813F
:1031800008958A3008F00895E82FF0E0E359FD4FE4
:1031900080810E9421150895CF93DF93CDE6D2E080
:1031A00089910E94591582E0C737D807C9F7DF9186
:1031B000CF91089590914E04982790934E0490914A
:1031C0004F04982790934F04909150049827909320
:1031D0005004909151049827909351049091520477
:1031E0009827909352040895AC0161157105A1F0E0
:1031F00020E0E0E0A0E0B0E0A40FB51F8C91E8274C
:10320000F0E0E454FD4FE0812F5FA22FB0E0A6175D
:10321000B70790F38E2F0895E0E0FCCF0E9474145E
:103220000E9475288823D1F30895EF92FF920F939F
:103230001F93CF93DF937C018B016115710561F0C2
:10324000C0E0D0E0F701EC0FFD1F80810E94CE01AD
:103250002196C017D107B0F3DF91CF911F910F9145
:10326000FF90EF90089522E42093E1041092E2048D
:1032700022E02093E3049093E4048093E504A1EE1C
:10328000B4E0E0E08D91E827F0E0E454FD4FE08108
:1032900084E0A63EB807B1F7EC93CD01059766E050
:1032A00070E00E941519089590E89093E10410923F
:1032B000E20421E02093E3048093E404ACEBB2E069
:1032C00090913C03FD01E90FF11D90819227FD01D2
:1032D000E90FF11D90819827A90FB11D8C91809362
:1032E000E50481EE94E065E070E00E941519089510
:1032F0001F920F920FB60F920BB60F921124DF920E
:10330000EF92FF920F931F932F933F934F935F93EF
:103310006F937F938F939F93AF93BF93CF93DF93DD
:10332000EF93FF931091CE008091BB02882309F4A4
:103330006EC080915B0490915C04895E934008F0BC
:1033400080C080915904803408F089C0282F2F5FF5
:10335000E82FF0E0EF5DFA4F1083209359041092AC
:103360005C0410925B04233008F451C07091210575
:103370009091220580E060912305462F50E0482B74
:10338000592B30E0CA0104962817390708F43FC0CA
:103390009A012D5F3F4FF901EF5DFA4F1081211522
:1033A000310509F401C190E0E0E0A0E0B0E0AF5DDC
:1033B000BA4F8C91E827F0E0E454FD4FE0819F5F25
:1033C000A92FB0E0A217B30790F31E1709F450C05D
:1033D0002115310509F4EAC090E0E0E0A0E0B0E09A
:1033E000AF5DBA4F8C91E827F0E0E454FD4FE081E7
:1033F0009F5FA92FB0E0A217B30790F38E2F90E044
:103400000E94AA011092590480E00E945419FF9171
:10341000EF91DF91CF91BF91AF919F918F917F916C
:103420006F915F914F913F912F911F910F91FF905D
:10343000EF90DF900F900BBE0F900FBE0F901F907C
:1034400018950E94E5150E9425171093210581E02B
:103450008093590410925C0410925B04D8CF0E94B0
:1034600054191092590410925C0410925B04CFCF4F
:10347000713809F492C17238B0F5713109F42BC179
:10348000723108F096C0713051F1703131F080E046
:103490000E94541910925904BACF6231C1F7809139
:1034A0002405082F10E0000F111F000F111F000F3F
:1034B000111F80912505080F111D02951295107F8F
:1034C0001027007F1027C6E2D5E08991B8010E943D
:1034D0006D1D0F5F1F4F85E0C633D807B1F781E040
:1034E0000E945419D7CF763809F435C1773808F0DF
:1034F00073C0723809F484C1753849F643305105F8
:1035000009F0A5C030912405932F80E02091250576
:10351000E22EFF24E82AF92AD0902605EAE3ED15E9
:1035200008F4B6CF7093E1041092E204F2E0DF0EEB
:10353000D092E3048EEFD80E3093E4042093E50498
:10354000DD2071F006EE14E0E701CE010E94B11D0E
:10355000F80181938F0121969E012E192D15A8F354
:103560008091E304682F6D5F09F4D5C1A1EEB4E04A
:1035700090E08E5F282F30E02E513B4F8D919827A1
:10358000E92FF0E0E454FD4F9081A217B307B1F7A3
:10359000E62FF0E0EF51FB4F90836F5F81EE94E0F8
:1035A00070E00E94151976CFE0E00FCF80E090E048
:1035B00027CF703409F453C1713409F068CF6230F9
:1035C00009F065CF9091240580E020912505820FB8
:1035D000911D0E94B4025ECF7738E9F1783809F086
:1035E00056CF7093E1041092E2048091240581305B
:1035F00009F46AC1813008F05BC180E18093E40482
:103600001092E5048093E6041092E70484E047E01A
:10361000A7E0B0E068E070E08093E30490E020E091
:1036200030E0F901EF51FB4F80819827E92FF0E05E
:10363000E454FD4F90812F5F3F4F241790F3AF511B
:10364000BB4F9C9381EE94E00E94151923CF80E03C
:103650000E9454191FCF80912405882309F006C1C8
:103660004230510509F014CFE0912505E43008F00F
:103670000ECF89E18093E1041092E20480E180930F
:10368000E3042E2F30E022953295307F3227207FC1
:103690003227A4EEB4E0F901E559F94F80818D930A
:1036A0002F5F3F4F84E0A43FB807A9F75397E0E0AE
:1036B0008D91E827F0E0E454FD4FE081F4E0A43F71
:1036C000BF07B1F7E093F404CD01439764E170E0E4
:1036D0000E941519DFCE623009F0D9CE8091240501
:1036E000082F10E0000F111F000F111F000F111FF6
:1036F00080912505080F111D02951295107F102746
:10370000007F102789E18093E1041092E20480E1B8
:103710008093E304C4EED4E0C8010E94B11D8993F4
:103720000F5F1F4F34E0C43FD307B1F7DE0153975B
:10373000E0E08D91E827F0E0E454FD4FE081CA1706
:10374000DB07B9F7E093F40481EE94E064E170E004
:103750000E9415199FCE9091240580E020912505A7
:10376000E22EFF24E82AF92A2EEFD22ED60E63503D
:103770006A3308F06CCFDD2009F4B1CE06E215E023
:10378000E701F80181918F01BE010E946D1D219614
:103790009E012E192D15A8F3A2CE87E190E09093FB
:1037A000E5048093E4048AEC90E09093E70480932E
:1037B000E604E4EBF2E0A8EEB4E081918D9322E020
:1037C000EA3BF207D1F781E88093E1041092E2042A
:1037D0008AE08093E304A1EEB4E0E0E08D91E82775
:1037E000F0E0E454FD4FE08134E0AE3EB307B1F7C2
:1037F000EC93CD010D976EE070E00E9415194ACE52
:103800004230510509F023CF30912405332309F4C8
:1038100068C09091250520E082E88093E104109231
:10382000E20483E08093E3043093E4049093E5049E
:103830002093E604A1EEB4E0E0E08D91E827F0E00B
:10384000E454FD4FE08184E0A73EB807B1F7EC9364
:10385000CD01069767E070E00E9415191BCE80919C
:103860007C0490917D040E94331914CE813009F0BC
:103870000ECE4231510509F00ACEE0912505E43023
:1038800008F005CE2E2F30E0A6E2B5E02295329565
:10389000307F3227207F32278D91F901E559F94F8A
:1038A00080832F5F3F4F85E0A633B807A9F717CE77
:1038B000883009F0ECCD81E08093E40444E0A4E09A
:1038C000B0E065E070E0A8CE88E08093E40480E199
:1038D0008093E50482E045E0A5E0B0E066E070E0BA
:1038E0009BCE90912505973860F4953870F4993106
:1038F00081F0993120F0892F8158823030F020E01A
:103900008BCF973821F09838D1F721E085CF24E08C
:1039100083CF20E181CF90E03BCE2C98803408F01B
:103920008FE3611160E4442349F090E0882349F07B
:10393000682B962B98B92C9A2D9A089590E8882395
:10394000B9F7962B98B90895882319F42D982C98D7
:103950000895469A2C9808959F92AF92BF92CF9265
:10396000DF92EF92FF920F931F93CF93DF930E940A
:10397000E51580919A040E94F3150E9474140E9428
:103980003C14CC24DD249924AA240E9474140E949F
:103990007528882309F07CC08C2D0E946F17C60102
:1039A000880F991F8C0D9D1DE82EEE0CEE0CB92C86
:1039B000B294BB0CBB0C80ECB82287E1E80EC0E0EF
:1039C000D0E009C0802F0E94DB12882319F52196D0
:1039D000CD30D10559F1FC2EFE01E454FC4F00819D
:1039E000802F0E94C512882369F31E2D1C0F812F82
:1039F0006A2D492D0E948D1C8B2D812B0E94B50EA6
:103A00008C2F0E94DC16AA24A394802F0E94DB1224
:103A10008823E9F28E2D8F0D8B290E94F40E8F2DB5
:103A20000E94E7162196CD30D105A9F68FE00E94BD
:103A3000C5128823D9F182E0C816D1040CF449C01C
:103A400085E10E94C512882351F080E0992009F495
:103A500081E0982E8823C9F181E00E94211586B16A
:103A600090E08F739070892B09F48FCF0E94F11230
:103A7000882309F48ACF80E00E94A41C0E940517C5
:103A8000AA240E9474140E947528882309F484CF04
:103A90000E946B0FDF91CF911F910F91FF90EF90DC
:103AA000DF90CF90BF90AF909F9008958EE00E94DE
:103AB000C512882329F28FEFC8168FEFD80609F4B4
:103AC000BFCF0894C108D108BBCF81E00E9459152F
:103AD000C6CF0894C11CD11CB3CF282FF89495E011
:103AE000289800000000000000009EBD0DB407FEF5
:103AF000FDCF00000000000000001EBC0DB407FE5A
:103B0000FDCF8EB5289A000000000000000080FD67
:103B1000E7CF28980000000086E08EBD0DB407FEB8
:103B2000FDCF00000000289A000000000000000007
:103B300028980000000082E08EBD0DB407FEFDCF86
:103B40007EBD0DB407FEFDCF6EBD0DB407FEFDCFEB
:103B50002EBD0DB407FEFDCF00000000289A78941A
:103B60000895382FF89425E0289800000000000000
:103B700000002EBD0DB407FEFDCF000000000000C8
:103B800000001EBC0DB407FEFDCF8EB5289A0000C4
:103B900000000000000080FDE7CF28980000000032
:103BA00083E08EBD0DB407FEFDCF9EBD0DB407FEB4
:103BB000FDCF3EBD0DB407FEFDCF000000001EBCD2
:103BC0000DB407FEFDCF8EB5289A78940895892FFD
:103BD0008F7184FD806E0895EF92FF920F931F9373
:103BE000FA01D90186958083862F90E08F709070BE
:103BF0009595879595958795959587958C93862F1F
:103C00008770F801808362956F70F70160831F9160
:103C10000F91FF90EF900895FC0130E022953295CE
:103C2000307F3227207F322720838081660F660F06
:103C3000660F640F6F70862B8083089580915D04FA
:103C4000882349F087FD0EC083E00E94211584E09F
:103C50000E945915089583E00E94591584E00E943E
:103C60005915089583E00E94591584E00E9421159A
:103C70000895962F803110F08FEF0895682F70E02F
:103C8000660F771F6F5F734F892F0E946D1D80E055
:103C900008959B01803120F5682F70E0FB01EE0F45
:103CA000FF1FE753FC4F8081918128173907A0F04F
:103CB000009749F08150660F771F6050744F0E9443
:103CC0006D1D80E0089580E0660F771F6050744F8F
:103CD0000E946D1D80E00895C901009759F7F3CF48
:103CE0008FEF0895803198F470E06050784F90E045
:103CF0000024969587950794969587950794982F15
:103D0000802D680F791F8CE06030780710F08FEFFE
:103D10000895842F0E946D1D80E00895EF92FF9218
:103D20000F931F93CF93DF93C82FD0E0CC0FDD1FED
:103D3000CC0FDD1FCC0FDD1FC60FD11DC05CDF4FC8
:103D4000CC0FDD1FC295D295D07FDC27C07FDC274A
:103D5000EE24FF248701000F111F0F591A4FF8019D
:103D600080819181892FBE010E946D1DF8018081A3
:103D700091812196BE010E946D1D0894E11CF11CE9
:103D80002196F0E1EF16F10429F7DF91CF911F9111
:103D90000F91FF90EF90089590E0880F991F8F5F2B
:103DA000934F0E94B11D90E008950F931F93082F29
:103DB00010E0000F111FC8018050944F0E94B11DE8
:103DC00090E0019607531C4FF80120813181821742
:103DD000930708F49C01C9011F910F9108958091E8
:103DE000D00480939205809192050E94D51E9093F5
:103DF0008D0580938C05809192050E94CC1E909336
:103E000094058093930520919305309194058091BA
:103E10008C0590918D052817390720F01092940594
:103E2000109293058091810590918205E091920511
:103E3000F0E0EE0FFF1FE753FC4F608171810E949D
:103E40008C4590938205809381050895803198F484
:103E500070E06050784F90E0002496958795079425
:103E6000969587950794982F802D680F791F8CE081
:103E70006030780710F08FEF0895CB010E94B11DDC
:103E80000895EF92FF920F931F93CF93DF93E090EB
:103E90008105F09082050894E11CF11C80E00E94ED
:103EA00004138823C9F400E080919505813029F13D
:103EB00080E00E94DB12882329F0809195058823F9
:103EC00009F0BFC0013009F4E7C0DF91CF911F9125
:103ED0000F91FF90EF90089581E0809395051092E7
:103EE0009105109290058093640482E20E94591516
:103EF00001E0809195058130D9F60E942214282F87
:103F00008823B9F0215080919005909191057C0112
:103F1000EE0CFF1CEE0CFF1CEE0CFF1C880F991F13
:103F2000E80EF91EE20EF11CF0929105E092900568
:103F300001E087E10E94C512882341F0E0909305DB
:103F4000F09094050894E11CF11C01E083E00E94CC
:103F5000C512882329F0E0908C05F0908D0501E0D2
:103F600089E00E94C512882309F0A2C089E00E945E
:103F7000DB12882309F0BAC08AE00E94C5128823A8
:103F800009F0A5C08AE00E94DB12882309F490CFD3
:103F90008CE10E945915E091920520918C05309199
:103FA0008D05F0E0EE0FFF1FE753FC4F80819181FC
:103FB0002817390708F07CCF80918C0590918D05EA
:103FC000019690938D0580938C0580919205609168
:103FD0008C0570918D050E94491E809192050E946A
:103FE000D51E90938D0580938C0560918C05709102
:103FF0008D056150704080918105909182058617F2
:104000009707D8F4EB01219701C0E901809192054F
:104010001C2F6C2F0E94261F482F809192051F5F36
:10402000612F0E94721E9E012150304080918105B7
:10403000909182058C179D0740F388E08093670478
:1040400037CF82E20E9421151092640410929505E8
:1040500081E08093670420919005309191052115AE
:104060003105A9F0E0919205F0E0EE0FFF1FE75354
:10407000FC4F808191818217930748F02150304096
:10408000309382052093810587E080936704109226
:104090003804013009F019CFC7010E94EB010093E9
:1040A0003804DF91CF911F910F91FF90EF90089509
:1040B0008BE10E9421151092910510929005E090DD
:1040C0008105F09082050894E11CF11C4FCF8CE132
:1040D0000E9421151092910510929005E0908105A3
:1040E000F09082050894E11CF11C4CCF8BE10E94FA
:1040F0005915C0918105D0918205219680918C053A
:1041000090918D05C817D90708F036CF8091920598
:104110001C2F6C2F0E94261F482F80919205115052
:10412000612F0E94721E219680918C0590918D05C1
:10413000C817D90758F380918C0590918D05019788
:1041400090938D0580938C058091920560918C05EC
:1041500070918D050E94491E809192050E94D51E86
:1041600090938D0580938C0588E08093670404CF3D
:10417000EF92FF920F931F938091D004809392054A
:10418000809192050E94D51E90938D0580938C0599
:10419000809192050E94CC1E909394058093930584
:1041A000209193053091940580918C0590918D0517
:1041B0002817390720F010929405109293058091EA
:1041C000810590918205E0919205F0E0EE0FFF1FCE
:1041D000E753FC4F608171810E948C45909382056A
:1041E000809381058091920560918105709182058F
:1041F0000E94261F80938905809192056091890510
:1042000040EE55E028E935E00AE915E0ECEAEE2E4B
:10421000E6E0FE2E0E94EC1D81E0809328060E94BD
:10422000A6288091AC068093B3061F910F91FF9052
:10423000EF900895AF92BF92CF92DF92EF92FF92EC
:104240000F931F93CF93DF93C82EDD24CC0CDD1C7E
:10425000CC0CDD1CCC0CDD1CC60ED11C80E490E027
:10426000C80ED91ECC0CDD1CC294D29410EFD12202
:10427000DC24C122DC24AA24BB24C6010E94B11D77
:10428000D82FC0E07501EE0CFF1CE1E6F5E0EE0E64
:10429000FF1EF701D183C08300811181C601019601
:1042A0000E94B11D90E0082B192BF70111830083A8
:1042B0000894A11CB11C82E090E0C80ED91E90E1C8
:1042C000A916B104D1F6DF91CF911F910F91FF9004
:1042D000EF90DF90CF90BF90AF90089510928B0534
:1042E00084E20E9459150E94D0150E945C1710921A
:1042F000260680E00E94A41C089510928A05109260
:1043000026061092830580E00E94A41C0E94D0150E
:104310000E945C170E943C1408958091870590913B
:104320008805682F677096958795969587959695D9
:1043300087958F700E947B2C60918705709188050E
:104340009B0140E050E0DA01C90180709078A070D4
:10435000B070892F9A2FAB2FBB2780936E04DA01A0
:10436000C90180709074A070B070892F9A2FAB2F04
:10437000BB2780936C042070307240705070232FE4
:10438000342F452F552720936D0410929B05872FBE
:104390008F7184FD806E089581E080938A0581E2AB
:1043A0000E94211510926C0480916C0480936D041E
:1043B00080916D0480936E041092830510922606FE
:1043C000809161059091620590938805809387059F
:1043D0008F5F9F4F89F010928F0510929B0510926E
:1043E0007A040E948D2180935D0480912F0480FDCA
:1043F000FCCF81E0809383050E94E515089581E05C
:1044000080938B0584E20E9421150E94E515089592
:10441000DF92EF92FF920F931F93809112078823F0
:1044200009F481C284E00E942A29109286058091B5
:10443000860580938505109295051092910510923E
:1044400090050E94B8208091C406609105074091B4
:104450002106209127060BE616E00E94B92B8091D9
:1044600021066091270640919A0520912806009127
:104470009E05E09098050E94141857E0D52E07C0BD
:10448000113009F4FBC00E94502B8823C9F00E9410
:1044900074141091AB061330D9F0143088F3143033
:1044A000D9F11D3081F781E00E941F308091AB0669
:1044B0008D3049F3109272040E94502B882339F7F3
:1044C0000E94322B0E9474141091AB06133029F70E
:1044D0000E943029882309F09CC10E94A22A8823C7
:1044E00021F010926404109272040E945A138823DF
:1044F00051F2182F11500E940517812F0E94DC16CF
:104500001093AC0680911207882309F0BCCF8091EC
:10451000AC068093B306B7CF0E943029882309F0F8
:104520005AC180919505882309F44AC10E94411F10
:1045300083E00E940413882309F03BC187E10E94B5
:104540000413882309F02EC186E10E9404138823F6
:1045500009F468C080912806882309F0AEC18091D3
:10456000AC068093B306E0908105F09082058091BF
:104570008605882309F08EC180912706882309F4D7
:104580004AC010E020910507309121068091B306C2
:1045900090E082959295907F9827807F98278093CE
:1045A000890580918905220F220F220F230F210FE9
:1045B0002F70282B209389058091920560918105A9
:1045C00070918205409189050E94721E1F5F809143
:1045D00081059091820501969093820580938105D3
:1045E0000894E11CF11C8091810590918205E09175
:1045F0009205F0E0EE0FFF1FE753FC4F60817181E1
:104600000E948C45909382058093810580912706B6
:10461000181708F4B7CF80918505882309F050C199
:10462000D092670480916704873009F405C18091B6
:104630006704883009F457C180916704813009F418
:10464000AEC08091AB06843011F01092720480915C
:104650001207882309F4D9C080917104813009F0D0
:1046600012CF109271040E947528882309F40BCF91
:104670001F910F91FF90EF90DF9008950E943029D5
:10468000882309F073C00E94411F83E00E94041335
:10469000882339F583E00E94DB128823F1F490919E
:1046A00092058091D004981711F00E94B820809153
:1046B000AB06813011F010927204809112078823AA
:1046C00009F0B6C00E947528882309F4DCCE1F913A
:1046D0000F91FF90EF90DF90089583E20E945915AB
:1046E000DECF109282051092810580919205609133
:1046F0008105709182050E94261F80938905809113
:1047000092056091890540EE55E028E935E00AE917
:1047100015E0ACEAEA2EA6E0FA2E0E94EC1D81E03C
:10472000809328068091AC068093B3060E94A62849
:104730008091C406609105074091210620912706CB
:104740000BE616E00E94B92B8091210660912706A6
:1047500040919A052091280600919E05E0909805C9
:104760000E94141883E20E94211594CF0E94D01554
:1047700082E20E9421151093720481E20E94591571
:10478000809121066091270640919A052091280684
:1047900000912106E09098050E94141874CF1092A1
:1047A00067044FCF81E08093860580E00E943D152D
:1047B000CBCE81E08093850583E20E943D15BECE7D
:1047C0000E941F2B8091920586958093DA0480E0E9
:1047D0000E941F30ABCE0E94D01582E20E942115AC
:1047E00081E08093720481E20E942115809121066C
:1047F0006091270640919A05209128060091210694
:10480000E09098050E9414188CCE81E00E942A291D
:1048100023CF0E94D01511E01093640484E20E941B
:1048200021158091AC060E94DC161093720455CEBF
:1048300084E00E942A2946CF8091920560918105EB
:10484000709182050E94261F8093890580919205B0
:104850006091890540EE55E028E935E00AE915E068
:104860009CEAE92E96E0F92E0E94EC1D11E01093CF
:104870002806809121066091270640919A05209193
:10488000280600919E05E09098050E941418109348
:104890006704D2CE10928605809192056E2D0E94FB
:1048A000391E809192050E94CC1E909394058093AE
:1048B000930580E00E9459155FCE0E94A6284FCE36
:1048C0001092850580919205B7010E94491E809142
:1048D00092050E94D51E90938D0580938C0583E2EE
:1048E0000E9459159DCE809192056091810570912D
:1048F00082050E94261F8093890580919205609110
:10490000890540EE55E028E935E00AE915E0BCEA02
:10491000EB2EB6E0FB2E0E94EC1D81E08093280672
:104920001092670489CE81E00E942A297ECDEF9201
:10493000FF920F931F9380911207882309F4AAC155
:1049400084E00E942A291092860580918605809332
:1049500085051092950510929105109290050E9480
:10496000B8208091C40660910507409121062091EE
:1049700027060BE616E00E94B92B80912106609174
:10498000270640919A052091280600919E05E09007
:1049900098050E94141808C0143009F45FC00E94E2
:1049A000502B882309F490C00E9474141091AB0618
:1049B000113091F70E943029882309F0DAC083E092
:1049C0000E940413882309F0F5C083E00E94DB12E3
:1049D000882309F039C180E00E940413882309F07C
:1049E0003CC180E00E94DB12882309F04BC190910A
:1049F00092058091D0049817E1F00E94B820809130
:104A0000C4066091050740912106209127060BE618
:104A100016E00E94B92B80912106609127064091F3
:104A20009A052091280600919E05E09098050E9425
:104A300014188091AB06813011F0109272048091AD
:104A40001207882309F043C00E947528882309F4BF
:104A5000A6CF1F910F91FF90EF9008950E943029EB
:104A6000882309F065C086E10E940413882309F0B9
:104A700053C083E00E940413882309F041C080E002
:104A80000E940413882339F580E00E94DB128823FA
:104A900079F58091AB06843011F010927204809108
:104AA0001207882309F461C080917104813009F0F4
:104AB00076CF109271040E947528882351F60E94C7
:104AC000502B882309F070CF0E94322B6DCF84E0E9
:104AD0000E942A29B9CF11E01093950582E20E9425
:104AE00059151093380480E00E94DB12882389F264
:104AF00082E20E9421151092950510923804C9CFC8
:104B000081E08093850583E20E942115109286053D
:104B100080E00E945915B3CF81E08093860580E044
:104B20000E9421151092850583E20E945915A1CF9C
:104B30000E94D01582E20E94211581E080937204C8
:104B400081E20E9421158091210660912706409103
:104B50009A052091280600912106E09098050E9470
:104B6000141881E00E9427027ECF81E00E942A294A
:104B70009BCF0E94D01582E20E94211510937204EF
:104B800081E20E945915809121066091270640918B
:104B90009A052091280600912106E09098050E9430
:104BA000141881E00E94270283E00E9404138823E6
:104BB00009F40BCF10928205109281058091920525
:104BC00060918105709182050E94261F809389055E
:104BD000809192056091890540EE55E028E935E025
:104BE0000AE915E07CEAE72E76E0F72E0E94EC1D3C
:104BF00081E0809328068091AC068093B3060E94E2
:104C0000A6288091C4066091050740912106209155
:104C100027060BE616E00E94B92B809121066091D1
:104C2000270640919A052091280600919E05E09064
:104C300098050E94141883E20E94211583E00E94C7
:104C4000DB12882309F4C7CE83E20E94591580E065
:104C50000E940413882309F4C4CE11E01093950533
:104C600082E20E94591580918105909182050196FA
:104C70000E94EB011093380480E00E94DB1288232D
:104C800009F4B5CE82E20E9421151092950510928A
:104C90003804ADCE81E00E942A2955CEEF920F93C1
:104CA0001F9310925F0480911207882309F419C2A0
:104CB00084E00E942A2910928605809186058093BF
:104CC00085051092950510929105109290050E940D
:104CD000EF1E07C0113009F48FC00E94502B8823AB
:104CE000C9F00E9474141091AB061330D9F014303F
:104CF00088F31430D9F11D3081F781E00E941F3014
:104D00008091AB068D3049F3109272040E94502BB3
:104D1000882339F70E94322B0E9474141091AB063D
:104D2000133029F70E943029882309F0B0C00E946F
:104D3000A22A882321F010926404109272040E9427
:104D40005A13882351F2182F11500E940517812FF2
:104D50000E94DC161093AC0680911207882309F09C
:104D6000BCCF8091AC068093B306B7CF0E943029A8
:104D7000882309F0D3C080919505882309F4C3C026
:104D800083E00E940413882329F080915F0481301E
:104D900009F483C187E10E940413882309F08CC0C1
:104DA00080E00E940413882309F092C080E00E94F2
:104DB000DB12882309F09AC08091AB06843011F091
:104DC0001092720480911207882309F46FC08091B9
:104DD0007104813009F081CF1092710480915F04D9
:104DE000882309F07ACF0E947528882309F475CFAB
:104DF0001F910F91EF9008950E943029882309F0A8
:104E0000D7C080919505882309F4F7C083E00E94FC
:104E10000413882379F081E080935F0480915F041C
:104E2000882309F42EC183E20E9421151092820585
:104E30001092810580E00E940413882309F0E8C0E5
:104E400010919505113009F4FBC080E00E94DB123F
:104E5000882309F087C0909192058091D00498171B
:104E600011F00E94EF1E8091AB06813011F010927C
:104E7000720480911207882309F4B5CF84E00E9460
:104E80002A290E947528882309F427CFB1CF0E94D0
:104E9000D01511E01093640484E20E9421158091E2
:104EA000AC060E94DC161093720441CF81E00E9490
:104EB0002A2910925F048BCF81E08093860580E0E1
:104EC0000E943D1580E00E940413882309F46ECFF0
:104ED00011E01093950582E20E9459151093380451
:104EE00080E00E94DB12882309F466CF82E20E94F0
:104EF00021151092950580913804813009F4E2C0A3
:104F00001092380459CF0E941F2B809192058695EC
:104F10008093DA0480E00E941F3032CF0E94D015C7
:104F200082E20E94211581E08093720481E20E9456
:104F30002115809121066091270640919A052091C4
:104F4000280600912106E09098050E94141880918F
:104F50005F04882309F499C083E20E943D150E94F2
:104F6000251709CF82E20E94211510929505209104
:104F70009005309191052115310591F0E091920550
:104F8000F0E0EE0FFF1FE753FC4F80819181821705
:104F9000930730F0215030403093820520938105F3
:104FA00080913804813009F47EC01092380453CFC8
:104FB0000E94D01582E20E9421151093720481E2B2
:104FC0000E945915809121066091270640919A050B
:104FD0002091280600912106E09098050E9414185F
:104FE00080915F04882309F454C083E20E94211554
:104FF00080919505882309F009CF0E941F2B80918D
:10500000920586958093DA0480E00E941F30FECEE0
:1050100011E010939505109291051092900582E28F
:105020000E945915809181059091820501960E94F8
:10503000EB011093380410919505113009F005CF5C
:105040000E942214482F882309F4FFCE415020915A
:10505000900530919105C901880F991F880F991FFC
:10506000880F991F220F331F820F931F840F911DEA
:1050700090939105809390050E94EB011093380462
:10508000E4CE83E20E945915D1CE83E20E945915E5
:1050900066CF83E20E945915B4CE8093850583E2E2
:1050A0000E94211577CE80912106609127064091BC
:1050B0009A052091280600912106E09098050E940B
:1050C000141873CF809121066091270640919A05AC
:1050D0002091280600912106E09098050E9414185E
:1050E0000FCF81E00E942A29E6CD9091CF048091D4
:1050F000D504891731F08091CF048093D50481E0E5
:10510000089580E0089580912806882391F0809189
:10511000E0058093C40680919805809305078091EF
:105120009A05809321068091280680932706109285
:10513000280680912706882329F0809127068093EE
:105140002706089581E08093270608958091E00561
:105150008093C406809198058093050780919A05F5
:1051600080932106809128068093270610922806B6
:105170000895833059F0843050F0843029F08091C4
:10518000AC068093B30608951092AC060895823061
:10519000B0F70895FC0187858F708D30C1F030E045
:1051A00020E190E080818F708E3061F09F5F3196BA
:1051B0009217C0F3892F913118F48150832B0895F1
:1051C00080E1FBCF9923B1F780E0832B089530E194
:1051D0002FE0E7CF1F93DF93CF930F92CDB7DEB7CA
:1051E000162F0E94CA28898389818F708F5F8093D0
:1051F000EB0310939E05898184FD08C086E08093AF
:10520000E9030F90CF91DF911F91089588E080937B
:10521000E9030F90CF91DF911F910895E82FF0E0FF
:10522000EF73F070E451FC4F8081089540939C052A
:105230006093DF058093AB0681E080932406089598
:10524000882339F08091DF058093AB0681E080935D
:10525000240608958093AB0681E080932406089588
:1052600080912406882319F01092240681E0089585
:105270003F924F925F926F927F928F929F92AF92E6
:10528000BF92CF92DF92EF92FF920F931F93CF9333
:10529000DF93462E4A015901662309F4C4C09C01DC
:1052A000E90100E0FF241FEFDD2466247724B2E04B
:1052B0005B2E33243394CE010E94CA28F301E155BA
:1052C000F94F8083C0802FE0C222C39440E050E0B9
:1052D00012C01E251F7BF1F4F501E00FF11D308295
:1052E000FF2009F070C0DD24D3940F5F4F5F5F4F44
:1052F0001E2D4C1588F5642FFE01E40FF51FE0808C
:105300002E2D30E0C9018F7090700F9709F455C0B1
:10531000DD20F9F6F501E00FF11D5082EF2DF0E0F0
:10532000D401AE0FBF1FEC926295607FE75DF94F2D
:105330006083F3940024220F331F001C220F331FBD
:10534000001C232F302DDD24D394D2220F5F4F5F1A
:105350005F4F1E2D4C1578F20894611C711C6096ED
:10536000641408F4A8CF003408F061C08F2DF50153
:10537000E00FF11D10820F5F0034C8F39FE39F150B
:1053800050F09FEFEF2DF0E0E75DF94F9083F3943D
:105390002FE32F15B8F7DF91CF911F910F91FF9059
:1053A000EF90DF90CF90BF90AF909F908F907F90C5
:1053B0006F905F904F903F900895F501E00FF11DC1
:1053C0001082DD2492CFEF2DF0E03197E80DF91D2A
:1053D000E082FA94EF2DF0E0F394E75DF94FA081BD
:1053E000AF70BA2FBF5F808182958F70682F70E099
:1053F000CB018B0F911D40970CF0BA2F0024220F88
:10540000331F001C220F331F001C232F302DDD24DF
:10541000D394D22262957295707F7627607F76272B
:10542000B62BB08362CF00E0FF2480E0A0CF8F2DA9
:10543000A5CF2F923F924F925F926F927F928F9261
:105440009F92AF92BF92CF92DF92EF92FF920F9313
:105450001F93CF93DF935C01562E3A0169016623B7
:1054600009F45DC0482EEC0130E060E0EE24FF243A
:10547000FA9480E000E010E05FE04EE0342E2DE092
:10548000222E9FEA892E96E0992E800E911EF4011D
:1054900070817F707F5FDE0190E0442D41950BC0ED
:1054A0005C93223089F0E42EEA0E3F5F9F5F1196F5
:1054B000822F9717D0F4F601E30FF11D20812130E0
:1054C00079F7882349F45C93F301E60FF11DF0802E
:1054D0006F5FFC9222E0E7CF5C93F501EE0DF11DCA
:1054E000808180648083FC92DECF903158F4FE018D
:1054F000E90FF11D30829F5F05C0FE01E90FF11D2C
:1055000050839F5F9031C8F3F401808184FD2F8622
:105510000F5F1F4F6096822F051508F4B2CFDF9101
:10552000CF911F910F91FF90EF90DF90CF90BF90A0
:10553000AF909F908F907F906F905F904F903F9033
:105540002F90089580919C050E94DB12882339F0EA
:105550008091DF058093AB0681E080932406089557
:1055600010928B0584E20E9459151092610480E02C
:105570000E9459150E945C170E9460160E94E51552
:105580008091D9040E94F31580E00E94A41C089524
:1055900081E080938B0584E20E9421150E94E5152D
:1055A00080E00E94F31580E00E94A41C08951092F0
:1055B00026060E9460160E94E5150E945C178091E5
:1055C000D9040E94F3151092220681E20E94591517
:1055D00080E00E94A41C109212078CEF0E941C0F06
:1055E000089510929B0581E08093220681E20E943B
:1055F000211580E00E94A41C80912E04882321F4B0
:1056000080912F0480FDFCCF10922F0410923E0455
:1056100010923D04109243041092450410924404E9
:1056200010928604809186048093880481E08093A0
:105630002606809312078AEF0E941C0F089588E0C7
:105640000E940413882369F09091AB0688E0809350
:105650009C059093DF0583E08093AB0681E0809307
:105660002406089580917204882311F480E008953F
:1056700081E00E940413882321F081E08093730469
:10568000089581E00E94C512882381F380E00E9482
:10569000AF12882359F382E08093730481E0089568
:1056A00080912E04823011F080E008950E944B0F0B
:1056B0008093070780E00895AF92BF92CF92DF9268
:1056C000EF92FF920F931F93CF93DF935B01C82E4E
:1056D000DD24C294D29450EFD522DC24C522DC24F0
:1056E000EE24C0E0D0E0FF24F39405C02196F394AB
:1056F000F1E1FF16B1F085010C0F1D1FC6018C0FE3
:105700009D1F0E94B11DF8018083EE2079F78081F2
:105710008F708E3059F7EF2C2196F394F1E1FF163C
:1057200051F7EE20A1F490E1F50187858F708D305F
:10573000B9F0892F81508F70DF91CF911F910F9118
:10574000FF90EF90DF90CF90BF90AF9008959E2D87
:10575000915051F791E0F50187858F708D3049F7B1
:10576000903110F08EE1E8CF892F81508F708061E9
:10577000E3CFBF92CF92DF92EF92FF920F931F93EE
:10578000CF93DF936801E82EFF24EE0CFF1CE60E9A
:10579000F11CEE0CFF1CEE0CFF1CEE0CFF1CE40ECB
:1057A000F11CE294F29470EFF722FE24E722FE242B
:1057B00030E022953295307F3227207F3227B22E7B
:1057C000222379F0C0E0D0E086010C0F1D1FC70135
:1057D0008C0F9D1F0E94B11DF80180832196CB156F
:1057E00098F3DF91CF911F910F91FF90EF90DF9091
:1057F000CF90BF900895EF92FF920F931F93CF9396
:10580000DF93182F062F0E942517E12EFF24EE0CA0
:10581000FF1CEE0CFF1CEE0CFF1CE00EF11CE294D2
:10582000F294A0EFFA22FE24EA22FE24C0E0D0E0A7
:10583000FE01EC54F94F8081BE016E0D7F1D0E9468
:105840006D1D2196C031D10599F70E942517DF9172
:10585000CF911F910F91FF90EF900895CF92DF921B
:10586000EF92FF920F931F93CF93DF93E22E680185
:10587000082F10E0000F111F060F111D000F111F40
:10588000000F111F000F111F040F111D029512951B
:10589000107F1027007F1027FF24E294F29480EFFE
:1058A000F822FE24E822FE24FE2C82E00E9421152C
:1058B0000E942517EE2089F0C0E0D0E0F601EC0F41
:1058C000FD1F8081B8016C0F7D1F0E946D1D84E05B
:1058D0000E94F60D2196CF1588F382E00E9459159B
:1058E0000E942517DF91CF911F910F91FF90EF90AC
:1058F000DF90CF900895EF92FF920F931F93CF9375
:10590000DF93182F062F0E942517E12EFF24EE0C9F
:10591000FF1CEE0CFF1CEE0CFF1CE00EF11CE294D1
:10592000F29440EFF422FE24E422FE24C0E0D0E012
:10593000CE018E0D9F1D0E94B11DFE01EC54F94F4A
:1059400080832196C031D10599F71092610480E0DF
:105950000E9476150E942517DF91CF911F910F911C
:10596000FF90EF90089580912E04882349F40E94BF
:10597000A50080912E04813049F00E9464120895A0
:105980000E94B00380912E048130B9F70E946B12FF
:1059900008959F92AF92BF92CF92DF92EF92FF92C3
:1059A0000F931F9381E08093AB068093240600E061
:1059B00011E032E0F32E2FE0E22E94E0D92E86E0C3
:1059C000C82EB7E0BB2EAAE0AA2EF0E29F2E0E94BE
:1059D00074148091AB06863009F46FC0873008F0EC
:1059E000AAC0813009F456C1843089F78091240619
:1059F000882339F0109224061093670410926504EE
:105A000000E080919C050E94DB12882331F1809197
:105A1000DF058093AB06109324060023E1F080910C
:105A20006504882311F41093650480916504813224
:105A300010F090926504909100028091650498178F
:105A400051F080916504809300026091000287E02C
:105A500090E00E945002109238040E942214282FD5
:105A6000882381F0809165048A9DC0011124809370
:105A70006504809165048150820F80936504F092E3
:105A8000670401E080916704882309F4A0CF909116
:105A9000000280916704823009F4FDC1892F90E0F3
:105AA0000E94EB0110933804109267040E94741452
:105AB0008091AB06863009F091CF8091240688232F
:105AC00039F010922406109267041092650400E0E9
:105AD00080919C050E94DB12882349F08091DF05AC
:105AE0008093AB0610932406002309F0D7C1809160
:105AF0006504882309F475C120916504213009F4F7
:105B000053C120916504223009F422C180916704B9
:105B1000813009F43EC180916704823009F057CF8B
:105B2000109267040E94E51580919A040E94F31573
:105B30000E9425174CCF873009F450C08F3009F0F0
:105B400046CF80912406882349F0109224061093B2
:105B500067048091D0048093660400E080919C05E6
:105B60000E94DB12882349F08091DF058093AB0609
:105B700010932406002309F068C10E94A81388230B
:105B800069F0982F9150933048F4809194049817BD
:105B900029F0909394041093670401E08091940499
:105BA000813009F436C180916704882309F40FCF4E
:105BB000109267040E94CE160E94E515809194040D
:105BC0008F5F0E946E1680919404813009F0FFCEA1
:105BD0008091970481500E94F315F9CE809124069C
:105BE000882321F0109224061093670480919C056D
:105BF0000E94DB12882351F08091DF058093AB0671
:105C0000109324068091670481FD31C10E94A8137E
:105C1000882389F0982F9150933068F480912E0456
:105C2000981749F090932E040E94B32C809167043A
:105C300083608093670483E00E94C512882379F013
:105C400080916A048F5F80936A0480916A048170F6
:105C500080936A04809167048360809367048091D5
:105C6000670480FFB4CE809167048E7F80936704C1
:105C70000E94CE1680912E048F5F0E946E1683E2E2
:105C80000E94591580916A04882309F414C10E9466
:105C900025179DCE80912406882331F0109224068A
:105CA0000E94D0150E94251787E10E9404138823C3
:105CB00059F09091AB0687E180939C059093DF05A6
:105CC000B092AB061093240688E00E940413882348
:105CD00059F09091AB0688E080939C059093DF0586
:105CE000C092AB061093240681E00E94041388231F
:105CF00051F08091AB0610939C058093DF05D09204
:105D0000AB06109324068EE00E940413882359F0FA
:105D10009091AB068EE080939C059093DF05E09216
:105D2000AB06109324069091CF048091D504891777
:105D300009F44DCE8091CF048093D5041F910F912B
:105D4000FF90EF90DF90CF90BF90AF909F9008951D
:105D50009091D00480916604981759F08091D004F6
:105D600080936604209367048091660480939A046C
:105D700001E089E00E94DB12882309F4C7CE10926B
:105D800065048BE10E94591580916704813009F008
:105D9000C2CE109267040E94E5158091AD040E9466
:105DA000F3150E94251713CE9091D00480916604BC
:105DB000981759F08091D00480936604209367046B
:105DC000809166048093AD0401E08AE00E94DB12BA
:105DD000882309F496CE109265048CE10E9459152F
:105DE00090CE8AE00E94C512882309F068C089E03D
:105DF0000E94C512882309F47FCE8BE10E942115F1
:105E0000F0926504F09267048091D0048093660458
:105E100073CE909166048091D004981709F4C3CE94
:105E20008091D00480936604909166049F5F9230C5
:105E300008F451C080919704981709F4B4CE909358
:105E400097041093670401E0AECE809197046091AF
:105E5000940490E0019782959295907F9827807F97
:105E60009827682B8AE090E00E94500286CE8091AD
:105E70006A0490E08170907082959295907F982747
:105E8000807F982760912E046F70682B82E090E0ED
:105E90000E945002BBCE9091650400CE83E090E05A
:105EA0006091AD040E94500284E090E060919A04F9
:105EB0000E9450021CCE83E20E942115E8CE8CE1A4
:105EC0000E94211510936504109367048091D004FB
:105ED000809366048CCF92E0ADCF1F93DF93CF9376
:105EE0000F92CDB7DEB71092120780E00E94A41C7B
:105EF0008CEF0E941C0F80912E04813011F00E94C3
:105F00003A1280912806882391F08091E0058093D1
:105F1000C406809198058093050780919A05809327
:105F200021068091280680932706109228069091DA
:105F3000980580910507981721F080919805809326
:105F4000050710926906109286048091860480935A
:105F50008804109299058BE696E09093AE068093A4
:105F6000AD06109121060E94CA28898389818F700D
:105F70008F5F8093EB0310939E05898184FD08C099
:105F800086E08093E9030F90CF91DF911F910895F0
:105F900088E08093E9030F90CF91DF911F910895DE
:105FA0001F93DF93CF930F92CDB7DEB780E00E94AF
:105FB000A41C1092690610922F0410923E041092B5
:105FC0003D04109243041092450410924404109230
:105FD0007404109286048091860480938804109241
:105FE00099058BE696E09093AE068093AD061091EE
:105FF00021060E94CA28898389818F708F5F8093D0
:10600000EB0310939E05898184FD17C086E0809381
:10601000E90383E0809312078AEF0E941C0F8091AE
:106020002E04813011F00E94381283E080933604F0
:106030000F90CF91DF911F91089588E0E8CFEF9204
:106040000F931F93982F882309F495C0813029F06E
:1060500080E01F910F91EF9008958091240688238E
:1060600009F0F9C00E94A813882399F1982F915044
:1060700080912806882341F48091210680939A0517
:106080008091C4068093E00580919A05891770F489
:1060900080919A05981B9F5F90932806809128060F
:1060A000853008F446C184E0809328068091120769
:1060B000882309F441C1809121066091270640910F
:1060C0009A052091280600919E05E09098050E946F
:1060D000141884E10E94C512882309F0DEC085E10E
:1060E0000E94C512882309F0CEC080911207882330
:1060F00021F590910507809198059817F1F080910E
:106100009805809305078091C4066091050740912A
:106110002106209127060BE616E00E94B92B8091FC
:1061200021066091270640919A052091280600914A
:106130009E05E09098050E9414188091120788230C
:1061400029F480912806882309F0D4C00E94C21344
:10615000982F882309F47CCF80916504915098177B
:1061600009F076CF8091DF058093AB0681E08093C4
:10617000240680E06ECF0E94A813982F8823D1F5C3
:1061800084E10E94C512882309F49FC010929805EB
:1061900088E00E94211581E00E9459158091120724
:1061A000882309F055CF909105078091980598179D
:1061B00009F44ECF80919805809305078091C4061D
:1061C0006091050740912106209127060BE616E015
:1061D0000E94B92B809121066091270640919A0573
:1061E0002091280600919E05E09098050E941418C1
:1061F00080E02FCF8091DA048093E00501E00093E6
:106200002806192F115010939A0584E10E94AF12AD
:10621000882309F44BC01092980588E00E9421154C
:1062200081E00E945915109365048091AB0680931C
:10623000DF058DE08093AB0681E080932406109209
:10624000AC0680911207882309F44FC081E01F91AA
:106250000F91EF900895109224069093720480910C
:1062600021066091270640919A0520912806009109
:106270009E05E09098050E9414180E94A813882398
:1062800009F427CFF3CE81E08093980588E00E943F
:10629000591581E00E94211528CF1092980588E0B9
:1062A0000E94211581E00E94591519CF85E10E94B5
:1062B000AF12882309F4B7CF0093980588E00E94B5
:1062C000591581E00E942115AECF85E10E94C512CB
:1062D000882309F463CF81E08093980588E00E94C9
:1062E000591581E00E94211559CF82E00E94B928FA
:1062F00081E0ADCF8091E0058093C4068091980540
:106300008093050780919A05809321068091280645
:1063100080932706109228068091C4066091050795
:1063200040912106209127060BE616E00E94B92B2A
:106330000DCF80912806B8CE8091E0058093C406E9
:10634000809198058093050780919A058093210696
:106350008091280680932706109228068091C40613
:106360006091050740912106209127060BE616E073
:106370000E94B92BA0CE2F923F924F925F926F92C4
:106380007F928F929F92AF92BF92CF92DF92EF92C5
:10639000FF920F931F93DF93CF930F92CDB7DEB78A
:1063A0000E9474141092AC068091AC068093B306E0
:1063B00080911207882311F40C944F3B84E0809362
:1063C000AB0681E080932406662499248824552412
:1063D0007724739438E0432E26E0322E93E0292E62
:1063E0000E9474141091AB061830D9F0193008F0DF
:1063F0004CC0153009F49EC4163008F096C0113018
:1064000009F431C2143009F40CC40E94502B8823C3
:1064100039F70E94322B0E9474141091AB06183089
:1064200029F780912406882349F0109224060E94BF
:10643000D01583E20E9421157092640480919C051E
:106440000E94DB128823A1F08091DF058093AB06C8
:1064500070922406109264048091C406609105072E
:1064600040912106209127060BE616E00E94B92BE9
:106470000E94A813882309F00FC50E94C213882325
:1064800021F281500E940C18C0CF1B3009F4DEC2EB
:106490001C30D0F5193009F485C21A3009F0B5CF97
:1064A000809124068823F9F01092240680E00E944F
:1064B00021150E9425178091C4066091050740911F
:1064C0002106209127060BE616E00E942E2C80E084
:1064D0000E9459150E94251784E08093AB067092A4
:1064E00024061092640480916704882339F084E0C4
:1064F0008093AB0670922406109267048091670423
:106500008F5F8093670481CF1C3009F47CC11D30FC
:1065100009F07BCF81E00E941F308091AB068D3067
:1065200009F473CF1092720470CF163009F4FCC0D6
:10653000173009F06ACF80912406882389F11092E0
:1065400024060E94D015609127068BE696E045EC64
:1065500056E02FE935E00E94382980E00E9421159D
:106560001092670489E0809365041092660480911C
:106570002706882391F020E0E22FF0E0E155F94F63
:106580009081809166048F5F9F70890F809366046D
:106590002F5F80912706281778F3662499245524C5
:1065A00080E00E940413882311F06624639488E03D
:1065B0000E940413882311F012E0612E87E10E94EB
:1065C0000413882311F0B3E06B2E809165048930A9
:1065D00009F4E7C680916504813009F4BCC6809156
:1065E0006504882309F491C580916504882329F006
:1065F00080916504807F09F45FC0109165048EE08E
:106600000E94C512882351F08091650480618093B7
:10661000650485E080936704F2E05F2E8FE00E94BE
:10662000C512882351F080916504806280936504CF
:1066300085E0809367045524539484E10E94C51239
:10664000882349F08091650480648093650485E027
:106650008093670455248EE00E94DB12882341F06A
:1066600080916504807E8093650484E08093670454
:106670008FE00E94DB12882341F080916504807DC9
:106680008093650484E08093670484E10E94DB12B8
:10669000882341F080916504807B8093650484E0C9
:1066A0008093670480916704853009F44EC580911A
:1066B0006704843009F460C580916504883009F46A
:1066C0003CC48091670490E083709070892B09F03E
:1066D0004CC4662009F499CE609127068BE696E0BB
:1066E00045EC56E02FE935E00E94192A8091C40656
:1066F0006091050740912106209127060BE616E0E0
:106700000E942E2C91E0691609F446C5E2E06E164F
:1067100009F474C0F3E06F1609F077CE87E0809338
:10672000AB067092240671CE809124068823D9F09E
:10673000109224060E94D015609127068BE696E001
:1067400045EC56E02FE935E00E94382984E20E94AA
:1067500021151092670410926604E3E6E093650445
:1067600066249924882480E00E940413882311F071
:106770006624639488E00E940413882311F082E069
:10678000682E80916504833609F41EC580916504E6
:10679000813009F428C580916504833009F486C5E9
:1067A00080916504882309F451C48091670490E0C6
:1067B00083709070892B09F019C4662009F425CEE6
:1067C000609127068BE696E045EC56E02FE935E030
:1067D0000E94192A8091C406609105074091210604
:1067E000209127060BE616E00E942E2C91E06916F8
:1067F00009F4D2C4E2E06E1609F007CE3092AB067F
:106800007092240602CE80912406882389F010928B
:1068100024069091620480912706981709F42CC6EB
:10682000709267048091DF058093AB067092240616
:1068300080919C050E94DB12882309F4E6CD8091AB
:10684000DF058093AB06709224068091670488234D
:1068500009F4B7C58DE00E94591582E00E945915D0
:106860000E942517D2CD809124068823E9F010924A
:10687000240680E00E9427020E94D01582E20E9436
:1068800021151093720481E20E945915809121060E
:106890006091270640919A052091280600912106D3
:1068A000E09098050E94141880E00E941F3080E05C
:1068B0000E94C512882329F085E08093AB06709270
:1068C000240683E00E94C512882351F08091AB0614
:1068D00020929C058093DF054092AB0670922406BF
:1068E00088E00E940413882321F03092AB06709256
:1068F000240687E10E940413882329F087E080930F
:10690000AB06709224068BE00E940413882359F092
:106910009091AB068BE080939C059093DF0580936C
:10692000AB06709224068DE00E940413882361F068
:106930009091AB068DE080939C059093DF059CE0E1
:106940009093AB06709224068091AB06813011F0D3
:106950001092720480911207882329F084E08093BA
:10696000AB06709224069091CF048091D5048917CC
:1069700009F44BCD8091CF048093D5040F90CF9133
:10698000DF911F910F91FF90EF90DF90CF90BF901C
:10699000AF909F908F907F906F905F904F903F90BF
:1069A0002F90089580912406882371F01092240678
:1069B00082E20E94591581E00E94A41C80E00E949E
:1069C000A41C80E00E9427029091650480919D059F
:1069D0009817C9F09090650480919D058093650497
:1069E00080916704833009F4AAC5809167048230DE
:1069F00050F080919705882331F4E0916504F0E030
:106A0000E156FA4F708286E10E94C512882329F070
:106A100080919705882309F450C5809167048330DD
:106A200009F4BFC386E10E94DB12882309F4EDCC90
:106A300080916704823009F0E8CC7092670480E0AE
:106A40000E94A41C82E00E945915DFCC809124068C
:106A5000882361F01092240682E20E9459158FE08B
:106A60000E9421150E9425171092670480919C05B1
:106A70000E94DB12882309F442C08091DF058093D5
:106A8000AB067092240680916704882391F580916B
:106A9000C406309105072091210690E0880F991FC8
:106AA000830F911D880F991F880F991F880F991FB9
:106AB000280F209363048091270680936204882323
:106AC000C1F090E0A0E0B0E0282F30E022953295B0
:106AD000307F3227207F3227FD01E559F94F808131
:106AE000AF51BA4F8C939F5FA92FB0E0A217B307A5
:106AF0009CF38FE00E9459158DE00E9459158DE09E
:106B00000E94C512882309F480CC809167048823F1
:106B100009F07BCC80916204882309F476CC7092D2
:106B200067048091C406209105071091210690E02A
:106B3000880F991F820F911D880F991F880F991F29
:106B4000880F991F180F80916304181709F45DCC02
:106B50008DE00E94211582E00E9421150E942517D8
:106B60006091630480912706882309F440C0C62EF3
:106B7000DD24C294D294A0EFDA22DC24CA22DC24E1
:106B8000A12EBB24A294B294F0EFBF22BA24AF226C
:106B9000BA24750100E010E0C6010E94B11D882EE4
:106BA0000559194FF8018083C7010E94B11DB60134
:106BB0000E946D1D882DB7010E946D1D84E00E940A
:106BC000F60D0894C11CD11C0894E11CF11C8E2DFB
:106BD0008A19082F10E08091270690E082959295FF
:106BE000907F9827807F982708171907ACF210919B
:106BF00021068BE696E00E94CA28898389818F70DE
:106C00008F5F8093EB0310939E05898184FD51C5AE
:106C100086E08093E90382E00E9459150E942517BF
:106C2000F4CB809124068823E9F0109224060E9478
:106C3000D01582E20E9421157092720481E20E94B6
:106C40002115809121066091270640919A05209197
:106C5000280600912106E09098050E94141881E012
:106C60000E94270283E00E940413882309F445C090
:106C700080912806882309F00DC490910507809122
:106C80009805981781F08091980580930507809169
:106C9000C4066091050740912106209127060BE666
:106CA00016E00E94B92B609127068BE696E045EC32
:106CB00056E02FE935E00E94382980E090E0FC01A1
:106CC000E156FA4F1082019680349105C1F782E0B7
:106CD0008093640410920807109266041092650471
:106CE00010926704109297057092690489E080936E
:106CF000AB067092240699249A948091AB06843056
:106D000011F01092720480911207882321F470927E
:106D1000AB067092240680917104813009F075CB26
:106D2000109271049091CF048091D504891709F0D5
:106D300021CE6BCB809124068823C9F010922406C3
:106D40000E94D015709267048BE696E00E94CA28D4
:106D5000282F2F702F5F2093650490E092958295E5
:106D60008F7089279F7089278170809366048EE0D9
:106D70000E944314823009F4D3C08AE00E94431475
:106D8000823009F4C4C089E00E944314823009F4BF
:106D9000B2C08FE00E94C512882399F02092670448
:106DA00080916604882319F49CE090936504809197
:106DB00066048F5F8093660480916604817080937F
:106DC00066048091670480FF21C080916704815030
:106DD0008093670480916604882309F4AAC1809196
:106DE0006504803108F4A8C381E08093650483E0E2
:106DF0000E94211580916504882309F097C181E0E4
:106E000080936504809165040E94FE1580E00E94D5
:106E1000DB12882309F4F9CA809167048230B8F143
:106E200082E0809364048BE696E061E045EC56E0F6
:106E30002FE935E00E94382990916504809166041D
:106E4000811180E191509F70892B8093AF068BE672
:106E500096E061E045EC56E02FE935E00E94192A02
:106E60008091C406609105074091210621E00BE660
:106E700016E00E942E2C8091C40660910507409177
:106E80002106209127060E94B92B1092640470926B
:106E9000AB0670922406B9CA182F1150812F0E9498
:106EA00004188091C40690910507E82EFF24EE0C8B
:106EB000FF1CE90EF11CEE0CFF1CEE0CFF1CEE0C8F
:106EC000FF1CE10EF11CE294F29450EFF522FE2437
:106ED000E522FE248701005F1F4F8FE0B7010E946B
:106EE0006D1D84E00E94F60D0894E11CF11CE01673
:106EF000F10699F7C2CA8091650490E00E968F70F2
:106F000090708F5F809365042092670442CF8091D8
:106F100065048F708F5F809365042092670433CF80
:106F200080916704823008F482C3809165048F5F8A
:106F3000809365042092670420CFE92DF0E0E156AC
:106F4000FA4F5082939480916604981610F066244C
:106F5000639470926704109265048091670490E0D6
:106F600083709070892B09F4B4CB0E94E515809151
:106F700027068823B1F090E080E001C08E2FE92F32
:106F8000F0E0E155F94FE081EF70EF5FE80F981600
:106F900018F09E1608F4DCC29F5F809127069817B0
:106FA00068F384E00E94591583E00E94591588E037
:106FB0000E9459158091670480FD13C0F2E05F16AE
:106FC00009F479C381E0581609F479C3552031F0EA
:106FD00084E00E94211583E00E94211588E00E9430
:106FE00021150E9425171092670473CB0E94E515A6
:106FF000E92DF0E0E75DF94F80818F3FD1F01081FE
:1070000012951F7000810F70010F0F5F101738F07D
:1070100010C0812F0E941C161F5F101750F4809122
:10702000670480FDF6CF812F0E94F3151F5F1017B4
:10703000B0F38091670480FFBFC1882D60E00E949B
:107040006F18109267040E942517B7CB86E10E9443
:10705000C512882309F0B8C20E945A13882309F088
:1070600081C287E10E94DB12882329F08FE3980E0A
:107070009822709267048EE00E94C512882321F046
:1070800090E1892A709267048FE00E94C5128823DC
:1070900021F0E0E28E2A7092670484E10E94C5121A
:1070A000882321F0F0E88F2A7092670485E10E941E
:1070B000C512882321F080E4882A709267048EE04C
:1070C0000E94DB12882321F09FEE892270926704D0
:1070D0008FE00E94DB12882321F0EFED8E22709268
:1070E000670484E10E94DB12882321F0FFE78F22EE
:1070F0007092670485E10E94DB12882309F455CB66
:107100008FEB88227092670450CB86E10E940413B3
:10711000882309F469CAE92DF0E0E156FA4F50805E
:107120007092650482E0809367045ECA8091650472
:1071300067CE80916504813108F4FBC181E08093C2
:10714000650483E00E94591555CE112309F0E8C16A
:1071500080916504882309F4E3C1662029F4E92DB0
:10716000F0E0E156FA4F508282E08093670480910C
:107170006704843009F0A0CA112359F08091650496
:10718000882339F4939480916604981610F066244D
:1071900063947092670490CA6092AB066092240672
:1071A00034C90E94F213882309F43CCC82E0809316
:1071B000670486E10E94AF12882309F033CC7092F5
:1071C00067040E94A41C2ECC88E00E94DB12882356
:1071D00009F4DCCA1092650470926704809165041A
:1071E000813009F0D8CA86E10E94DB12882309F0B9
:1071F00023C28EE00E94C512882349F0882D809515
:107200008071FFEE8F22882A82E0809367048FE0EE
:107210000E94C512882349F0882D809580729FEDC9
:107220008922882A82E08093670484E10E94C51243
:10723000882349F0882D80958078EFE78E22882A70
:1072400082E08093670485E10E94C512882349F09B
:10725000882D80958074FFEB8F22882A82E08093AE
:1072600067040E945A13182F882309F494CA80E0F7
:107270000E94A41C85E00E94F60D11501F7080EF43
:107280008822812AE82DF0E0EF73F070E451FC4F82
:10729000482D4078808160E00E948D1C82E08093C0
:1072A000670480916504833009F07ACA0E945A13FA
:1072B000182F0E947413882319F4112309F470CA3B
:1072C000E92DF0E0EB53F94F808280E00E94A41C8E
:1072D00085E00E94F60D93949FE3991518F410929F
:1072E000660499247092670410926504112309F4CE
:1072F00057CA812E8A94EFE08E228EE00E94AF1250
:10730000882311F0F0E18F2A8FE00E94AF128823CA
:1073100011F080E2882A84E10E94AF12882311F0E4
:1073200090E8892A85E10E94AF12882311F0E0E4F9
:107330008E2AE82DF0E0EF73F070E451FC4F482DF9
:107340004078808160E00E948D1C82E08093670419
:107350002092650425CA86E10E94DB12882311F081
:10736000409265048EE00E94C512882329F082E0D5
:1073700080936704A2E05A2E8FE00E94C5128823F2
:1073800029F082E0809367045524539484E10E949D
:10739000C512882309F423C982E080936704552429
:1073A0001EC987E10E94DB12882309F413C91092D9
:1073B0006504709267040EC9882D61E00E946F1801
:1073C00040CE82E00E9421150E9425179091C406AC
:1073D0002091050730912106809162048823B9F13C
:1073E000E92EFF24EE0CFF1CE20EF11CEE0CFF1C3C
:1073F000EE0CFF1CEE0CFF1CE30EF11CE294F29469
:1074000050EFF522FE24E522FE248701A0E0B0E043
:10741000FD01EF51FA4F8081A559B94F8C93B80106
:107420000E946D1D84E00E94F60D0F5F1F4F802F9C
:107430008E19A82FB0E08091620490E08295929519
:10744000907F9827807F9827A817B9070CF3109191
:1074500021068BE696E00E94CA28898389818F7075
:107460008F5F8093EB0310939E05898184FDE2C0BA
:1074700086E08093E903EEC9992309F4D1C982E239
:107480000E9459158DE00E9421150E942517109227
:107490006704CEC98091E0058093C4068091980569
:1074A0008093050780919A05809321068091280694
:1074B0008093270610922806EACB82E08093670427
:1074C0000E94DC13882311F020926704E091650488
:1074D000F0E0E156FA4F82E08083E0916604F0E04C
:1074E000EB53F94F808080922506E82DF0E0EF7392
:1074F000F070E451FC4F482D4078808160E00E949C
:107500008D1C80916504981639F0909065048091E7
:1075100066048F5F8093660482E00E9421157DCA15
:10752000939480916604981608F417CE66246394A9
:107530001BCE8091650403CE8091650456CC0E94D9
:10754000DC13882309F051CA82E0809367044DCA96
:10755000992D981B8091670480FF9DC0892F0E9400
:107560001C161FCD882E8A94FFE08F228EE00E9489
:10757000AF12882311F080E1882A8FE00E94AF12B9
:10758000882311F090E2892A84E10E94AF128823B7
:1075900011F0E0E88E2A85E10E94AF12882311F0F5
:1075A000F0E48F2AE82DF0E0EF73F070E451FC4F27
:1075B000482D4078808160E00E948D1C82E080939D
:1075C0006704209265044DCDE92DF0E0EB53F94FAF
:1075D00080808EE00E94AF12882311F0F0E18F2AA4
:1075E0008FE00E94AF12882311F080E2882A84E1A4
:1075F0000E94AF12882311F090E8892A85E10E9449
:10760000AF12882311F0E0E48E2AE82DF0E0EF734A
:10761000F070E451FC4F482D4078808160E00E947A
:107620008D1C82E0809367047092650415CD1092E2
:1076300065047BCC88E01DCFE92DF0E0EB53F94FDA
:1076400080828EE00E94AF12882381F588248FE02B
:107650000E94AF12882311F0F0E28F2A84E10E9489
:10766000AF12882311F080E8882A85E10E94AF12CA
:10767000882311F090E4892A80E00E94A41C93944E
:10768000EFE3E91518F410926604992470926704E8
:1076900010926504AECD892F0E94F31582CC81E053
:1076A0008093AB06809324060C94E43100E1802E95
:1076B000CECF88E0AECA84E00E94211592CC83E050
:1076C0000E9421158ECC0F931F93CF93DF93EC0173
:1076D000442319F18B0150E070E020E030E0F90123
:1076E000E155F94F60816F706F5FD80190E0FE0146
:1076F000E50FF11D80818D939F5F5F5F9617B8F353
:10770000760F2F5F3F4F005F1F4F241740F3872FE7
:10771000DF91CF911F910F91089570E0872FDF9136
:10772000CF911F910F910895BF92CF92DF92EF9268
:10773000FF920F931F93CF93DF936B01B42E4423DB
:1077400069F17C0110E000E0C0E0D0E0C7010E94D8
:10775000CA28FE01E155F94F808320812F702F5FE9
:10776000D70190E08D91F601E10FF11D80839F5FBD
:107770001F5F9217B8F3020F219680E190E0E80EA8
:10778000F91ECB1518F3802FDF91CF911F910F9128
:10779000FF90EF90DF90CF90BF90089500E0F3CF7F
:1077A000CF92DF92EF92FF920F931F93DF93CF93CD
:1077B000CDB7DEB7C054D0400FB6F894DEBF0FBED1
:1077C000CDBF109267041092650482E08093640438
:1077D000409127068BE696E06E010894C11CD11CEF
:1077E000B6010E94943BE82E809166048E1510F03D
:1077F00010926604809127068823C1F090E030E063
:10780000E32FF0E0E155F94F20812F702F5F80E0EA
:10781000E92FF0E0E75DF94F80838F5F9F5F82176C
:10782000B8F33F5F80912706381750F30E94741415
:1078300080911207882309F4C5C184E00E942A2997
:10784000FF240E9474141091AB06113071F01430B3
:10785000E1F10E94502B8823A1F70E94322B0E9455
:1078600074141091AB06113091F70E9430298823CF
:1078700009F0F4C086E10E940413882329F0809166
:107880006804882309F088C18091AB06813011F02B
:107890001092720480911207882309F070C10E942F
:1078A00075288823B1F210926404C05CDF4F0FB6D4
:1078B000F894DEBF0FBECDBFCF91DF911F910F9126
:1078C000FF90EF90DF90CF9008950E943029882399
:1078D00009F037C110E086E10E940413882309F003
:1078E000D0C087E10E940413882309F0E6C086E136
:1078F0000E94DB12882309F0FCC087E10E94DB12A2
:10790000882309F001C186E10E94C512882309F08D
:1079100006C18EE00E94C512882339F08F2D809514
:1079200080719FEEF922F82A12E08FE00E94C512C2
:10793000882339F08F2D809580729FEDF922F82AE7
:1079400012E084E10E94C512882339F08F2D8095C2
:1079500080789FE7F922F82A12E085E10E94C5129B
:10796000882339F08F2D809580749FEBF922F82AB7
:1079700012E00E945A13282F882361F08F2D90E087
:107980008F7090700D9734F421502F7080EFF82293
:10799000F22A12E088E00E94C512882309F44AC046
:1079A0008F2D90E08F7090700D970CF4ECC090EFDD
:1079B000F92200E010E080916604F601E80FF11D65
:1079C000F08240912706C6016BE676E00E94633B99
:1079D000E82E81E0809368040D301105BCF58F2DF1
:1079E00061E00E946F1884E20E9421150E94E51553
:1079F000E0916604F0E0E75DF94F80810E94F315A5
:107A00000E9425178091AB06843011F01092720409
:107A100080911207882309F4AEC0809171048130EF
:107A200009F017CF109271040E947528882309F479
:107A300010CF39CF123009F4C9C0113019F70F2D0A
:107A400010E00F7010700D3011054CF28F2D60E0BA
:107A50000E946F1884E20E945915C8CF0E94D01569
:107A600082E20E9421151093720481E20E9459154E
:107A700080916804882309F4A1C082E00E943D152A
:107A8000F9CE809166048F5F8093660480916604CE
:107A90006E2D0E9480459093660480916604F601E5
:107AA000E80FF11DF08082E00E94211511E087E1CE
:107AB0000E940413882309F41ACF809166046E2D66
:107AC00070E090E00197860F971F0E94A045809379
:107AD000660480916604F601E80FF11DF08080E0F5
:107AE0000E94211511E086E10E94DB12882309F42F
:107AF00004CF82E00E9459150E94251787E10E9459
:107B0000DB12882309F4FFCE80E00E9459150E9401
:107B1000251786E10E94C512882309F4FACE80E079
:107B20000E94AF12882309F4F4CE80919D058093C2
:107B3000660480916604F601E80FF11DF08011E003
:107B4000E8CE0E94D01582E20E94211581E0809348
:107B5000720481E20E942115809168048823C1F09B
:107B600082E00E943D1580916604F601E80FF11D48
:107B7000F08011E0B0CE81E00E942A294ECF84E04F
:107B80000E942A298CCE8FE0F82E0FE010E013CF50
:107B900082E00E945915E7CF82E00E94591580913A
:107BA000C4066091050740912106209127060BE647
:107BB00016E00E942E2C1092680466CE82E00E948D
:107BC000591558CE81E00E942A293ACE0F2D10E097
:107BD0000F701070F0CE3F924F925F926F927F9233
:107BE0008F929F92AF92BF92CF92DF92EF92FF92CD
:107BF0000F931F93DF93CF93CDB7DEB7C058D0401C
:107C00000FB6F894DEBF0FBECDBF1092670410927E
:107C1000650482E08093640440912706B1E4CB2E92
:107C2000D12CCC0EDD1E8BE696E0B6010E94943B73
:107C3000E82E0E94741480911207882309F42CC640
:107C400084E00E942A299924442488245524AA24C3
:107C5000AA94BB24332433943E010894611C711C04
:107C60000E9474141091AB061F30A9F0103108F077
:107C700088C0113009F4B8C2143009F44CC20E9413
:107C8000502B882369F70E94322B0E9474141091A4
:107C9000AB061F3059F70E943029882309F09BC496
:107CA0000E94A22A86E10E94C512882309F08AC494
:107CB00089E00E94C512882309F0D5C28AE00E949B
:107CC000C512882309F0C7C286E10E94DB1288230F
:107CD00009F0BDC289E00E94DB12882309F0B3C21B
:107CE0008AE00E94DB12882309F0A9C28DE00E947D
:107CF000C512882329F080916204882309F031C5D8
:107D000091E0991609F4DBC3A2E09A1609F4D3C3F3
:107D1000B3E09B1609F0B3CF30926804682D70E091
:107D2000842D992787FD9095860F971F850D911DAE
:107D30000E94A045582EEE2099F020E030E0F60198
:107D4000E20FF31F852D820F682D0E948045D3011D
:107D5000A90FB11D8C9180832F5F3F4F2E1578F3B3
:107D600040912706C6016BE676E00E94633B409196
:107D700027068BE696E0B6010E94943BE82E9924F4
:107D80007ECF113109F41BC1113108F480C01231CA
:107D900009F075CF0E943029882309F056C40E944B
:107DA000A22A8CE00E94C512882309F077C38CE0D8
:107DB0000E94DB12882309F06DC38EE00E94C51279
:107DC000882309F05DC38FE00E94C512882309F063
:107DD0004DC384E10E94C512882309F03DC385E1AB
:107DE0000E94C512882309F02DC388E00E94C512A5
:107DF000882309F01DC38EE00E94DB12882309F05E
:107E0000EFC28FE00E94DB12882309F0F2C284E106
:107E10000E94DB12882309F0F5C285E10E94DB1283
:107E2000882309F0F8C288E00E94DB12882309F059
:107E3000FBC2992009F423CF30926804EE2009F4A4
:107E40008FCF860110C00E97F9F08F2D8A21D801AF
:107E50009C919B21892BF80181938F018E2F8C1986
:107E60008E1508F07DCF0E94E000F82E90E08F7014
:107E700090708D30910539F7E7EFFE228F2D90E05D
:107E80008F7090700E9709F7F7EFFF22DECF0E94F8
:107E90003029882309F09EC20E94A22A8CE00E9409
:107EA000C512882309F0E7C187E10E94C512882323
:107EB00009F0ECC180E00E94C512882309F0F1C1ED
:107EC0008CE00E94DB12882309F0F6C187E10E9452
:107ED000DB12882309F0F9C180E00E94DB128823BD
:107EE00009F0FCC18EE00E94C512882309F0FFC191
:107EF0008FE00E94C512882309F008C284E10E9425
:107F0000C512882309F011C285E10E94C512882399
:107F100009F01AC288E00E94C512882309F023C222
:107F20008EE00E94DB12882309F02CC28FE00E94B1
:107F3000DB12882309F02FC284E10E94DB12882320
:107F400009F032C285E10E94DB12882309F035C2B4
:107F500088E00E94DB12882309F038C2992009F4D6
:107F60008ECE30926804E2E09E1609F4D0C3F4E0AD
:107F70009F1609F446C4B1E09B1609F003C4EE2035
:107F800009F4EECE860107C00F5F1F4F802F8C19BA
:107F90008E1508F0E5CE0E94E000F82EEFE1E8171C
:107FA00098F30E94E000D8012C916E2D0E9480452C
:107FB000F601E90FF11D80818C932083E5CF0E94AB
:107FC0003029882309F0F9C20E94A22A8CE00E947D
:107FD000C512882309F0E8C28CE00E94DB128823D6
:107FE00009F0DEC28EE00E94C512882309F0CEC2DD
:107FF0008FE00E94C512882309F0BEC284E10E946E
:10800000C512882309F0AEC285E10E94C5128823FB
:1080100009F09EC288E00E94C512882309F08EC232
:108020008EE00E94DB12882309F084C28FE00E9458
:10803000DB12882309F05FC284E10E94DB128823EF
:1080400009F062C285E10E94DB12882309F065C253
:1080500088E00E94DB12882309F068C28DE00E944C
:10806000C512882329F080916204882309F043C057
:10807000192D10FF04CE3092680411FDEFC2EE20DE
:1080800041F1860106C00F5F1F4F802F8C198E159E
:1080900000F50E94E000F82EBFE3B817A0F30E949D
:1080A000E000F82E90E08F7090708D30910509F40B
:1080B00004C30E9709F4FEC29F2D9A21D8018C911A
:1080C0008B21982B9C930F5F1F4F802F8C198E153F
:1080D00000F3BEEF9B2240912706C6016BE676E0D7
:1080E0000E94633B409127068BE696E0B6010E9412
:1080F000943BE82EC4CD892D80958270B1E09B22FF
:10810000982A8DE00E945915192D91FCA2C388244C
:108110000E942517AECF0E943029882309F07FC224
:1081200084E00E940413882309F072C285E00E9453
:108130000413882309F065C282E10E940413882396
:1081400009F058C281E10E940413882309F04BC250
:1081500086E10E940413882329F080916804882313
:1081600009F0EDC287E10E940413882329F0809171
:108170006804882309F0B2C28091AB06843041F0D4
:108180001092720482E00E94591582E20E945915F1
:1081900080911207882309F48AC18091710481308B
:1081A00009F06DCD109271040E947528882309F49E
:1081B00066CD10926404C058DF4F0FB6F894DEBF4E
:1081C0000FBECDBFCF91DF911F910F91FF90EF9028
:1081D000DF90CF90BF90AF909F908F907F906F90E7
:1081E0005F904F903F9008950E943029882389F432
:1081F0008091AB06813011F01092720480911207C9
:10820000882309F027C20E947528882309F437CDF6
:10821000D0CF0E94D01582E20E94211510937204E3
:1082200081E20E94591580916804882309F4A6C24E
:1082300082E00E943D1581E00E942702D9CF8CE1A7
:108240000E94591553CD8BE10E94591549CD82E00A
:108250000E9459153FCD8CE10E9421159F2C9394CB
:108260004424439431CD8BE10E9421159F2C93949B
:1082700044244A9423CD8EE00E942115992493949E
:1082800087E10E94C512882309F414CE80E00E9481
:108290002115F2E09F2E80E00E94C512882309F488
:1082A0000FCE82E20E942115E3E09E2E8CE00E9418
:1082B000DB12882309F40ACE8EE00E94591587E16B
:1082C0000E94DB12882309F407CE80E00E94591532
:1082D00080E00E94DB12882309F404CE82E20E942F
:1082E00059158EE00E94C512882309F401CE84E05E
:1082F0000E94211574E0972E60E1A62E5FEEB52E48
:108300008FE00E94C512882309F4F8CD83E00E9413
:10831000211544E0942E30E2A32E2FEDB22E84E1FD
:108320000E94C512882309F4EFCD88E00E94211530
:1083300094E0992E80E8A82E0FE7B02E85E10E94E8
:10834000C512882309F4E6CD81E00E94211514E0CE
:10835000912EB0E4AB2EAFEBBA2E88E00E94C5128E
:10836000882309F4DDCD84E20E942115F4E09F2EDC
:10837000EFE0AE2E70EFB72E8EE00E94DB12882366
:1083800009F4D4CD84E00E9459158FE00E94DB12DD
:10839000882309F4D1CD83E00E94591584E10E941D
:1083A000DB12882309F4CECD88E00E94591585E1BF
:1083B0000E94DB12882309F4CBCD81E00E9459157D
:1083C00088E00E94DB12882309F4C8CD84E20E9471
:1083D0005915C4CD89E10E942115992444245CCD0E
:1083E00084E00E9459158FE00E94DB12882309F473
:1083F0000ECD83E00E94591584E10E94DB12882390
:1084000009F40BCD88E00E94591585E10E94DB122A
:10841000882309F408CD81E00E94591588E00E9464
:10842000DB12882309F405CD84E20E94591501CDA1
:1084300084E20E942115992493942FE0A22E90EFBC
:10844000B92ED9CC81E00E9421159924939440E45F
:10845000A42E3FEBB32EC9CC88E00E9421159924AD
:10846000939460E8A62E5FE7B52EB9CC83E00E9416
:10847000211599249394E0E2AE2E7FEDB72EA9CC7E
:1084800084E00E94211599249394A0E1AA2EFFEE86
:10849000BF2E99CC8EE00E9459158FCC8EE00E94A1
:1084A000211599249394AA24AA94BB2480CC81E01A
:1084B0000E942A2972CE442009F02ECCE0CB442021
:1084C00009F4DDCB90926804EE2089F0342D3E0D46
:1084D000D60120E0822F830F6E2D0E948045F3018C
:1084E000E90FF11D8D9180832F5F2E1598F3409138
:1084F0002706C30138CC83E00E94591584E10E940D
:10850000DB12882309F49ECD88E00E94591585E18D
:108510000E94DB12882309F49BCD81E00E9459154B
:1085200088E00E94DB12882309F498CD84E20E943F
:10853000591594CD84E00E94591578CD84E20E94AB
:108540002115A1E09A2A1FE0A12EB0EFBB2E68CD25
:1085500081E00E94211591E0992A80E4A82E0FEB7A
:10856000B02E58CD88E00E94211581E0982A20E89D
:10857000A22E9FE7B92E48CD83E00E942115F1E09D
:108580009F2A40E2A42E3FEDB32E38CD84E00E9416
:108590002115E1E09E2A60E1A62E5FEEB52E28CDE2
:1085A0008EE00E9459151ECD8EE00E942115B1E08B
:1085B0009B2AAA24AA94BB240FCD8CE00E942115EB
:1085C000992402CD82E00E94211540909D0541949E
:1085D000992493946DCB80E20E9421159924442420
:1085E000FF2455245DCB6091AB0681E141E10E94FF
:1085F0001629AECD6091AB0682E142E10E941629B8
:10860000A1CD6091AB0680E145E00E94162994CD92
:108610006091AB068FE044E00E94162987CD0E944E
:10862000D01582E20E9421153092720481E20E94EC
:10863000211580916804882309F47DC082E00E949E
:108640003D1581E00E9427026BCD8BE00E94211531
:108650009924A5CB84E00E942A29D5CDEE2009F4E7
:1086600038CD860107C00F5F1F4F802F8C198E15E4
:1086700008F02FCD0E94E000F82EEFE3E81798F302
:108680000E94E000682D0E948045F301E90FF11D72
:10869000F0808F2D90E08F7090708D309105B9F043
:1086A0000E9791F09F2D9A21D8018C918B21982BB8
:1086B0009C93D9CFF7EFFF22FFCCE7EFFE228F2D5F
:1086C00090E08F709070F5CC87EFF822EBCFF7EF4A
:1086D000FF228F2D90E08F709070E2CF82E00E9499
:1086E00059158091C406609105074091210620919B
:1086F00027060BE616E00E94B92B40912706C80119
:10870000B6010E94943BE82E1092680435CD8E2D60
:10871000869509F425CBD6016E2D6150262F281B96
:108720008C91F601E60FF11D90819D93808361503D
:108730006217B1F715CB82E00E94591582CF82E013
:108740000E9459158091C406609105074091210649
:10875000209127060BE616E00E942E2C109268044A
:1087600001CDF39481E0F8228DE00E945915FF209D
:1087700009F07BC088240E942517C2CA82E00E94AB
:10878000591559CD609127068BE696E0A6012FE991
:1087900035E00E943829E82E882311F1860106C0B1
:1087A0000F5F1F4F802F8C198E15D0F40E94E000B0
:1087B000F82EBFE3B817A0F30E94E000F801208173
:1087C0006E2D0E948045F601E90FF11D8081D801D0
:1087D0008C9320830F5F1F4F802F8C198E1530F3E1
:1087E000609127068BE696E0A6012FE935E00E940E
:1087F000192A409127068BE696E0B6010E94943B29
:10880000AFCAEE2009F4ACCA860107C00F5F1F4F44
:10881000802F8C198E1508F0A3CA0E94E000F82E54
:108820008FE38F1598F30E94E000D8012C916E2DF4
:108830000E948045F601E90FF11D80818A219B2D60
:108840009223892B8C9380818B212A21822B8083F8
:10885000DDCF8DE00E94211581EE95E0B3014091BE
:1088600062040E94943B882E53CC8DE00E94211517
:1088700081EE95E0B301409162040E94943B882E02
:10888000409127068BE696E0B6010E94943BE82EC5
:10889000A3E09A2E44246FCF81E00E942A29D3C9F5
:1088A000EF92FF920F931F930E947414809112070E
:1088B000882309F421C184E00E942A29FF24F3942B
:1088C00007C0113009F471C00E94502B8823C9F0F1
:1088D0000E9474141091AB061330D9F0143088F351
:1088E0001430E9F11D3081F781E00E941F30809142
:1088F000AB068D3049F3109272040E94502B8823EE
:1089000039F70E94322B0E9474141091AB06133079
:1089100029F70E943029882309F092C00E94A22AD8
:10892000882321F010926404109272040E945A135A
:10893000882309F072C080911207882329F686E106
:108940000E94C512882309F0CCC086E10E94DB1288
:10895000882309F4B9CF80E00E94A41CB5CF0E94FF
:108960003029882309F081C080E00E941F300E94D6
:108970001F2B8091AB06843011F01092720480910D
:108980001207882309F46DC080917104813009F0C9
:108990009BCF109271040E947528882309F494CF0C
:1089A0001F910F91FF90EF9008950E943029882326
:1089B00009F077C080E00E941F3086E10E94C51256
:1089C000882301F586E10E94DB128823B9F40E9416
:1089D0001F2B8091AB06813011F0109272048091B0
:1089E0001207882309F079C00E947528882309F4AA
:1089F0006BCF1F910F91FF90EF90089580E00E9440
:108A0000A41CE5CF80E00E940E299091B306890F47
:108A100060E040E00E948D1CD5CF182F11500E94BD
:108A20000517812F0E94DC161093AC068091120767
:108A3000882309F080CF8091AC068093B3067BCF6A
:108A40000E94D015F092640481E00E94270284E223
:108A50000E9421158091AC060E94DC16F0927204EF
:108A60005DCF81E00E942A298FCF0E94D01582E23B
:108A70000E942115F092720481E20E9421158091DA
:108A800021066091270640919A05209128060091C1
:108A90002106E09098050E94141881E00E942702A8
:108AA00063CF0E94D01582E20E94211510937204B8
:108AB00081E20E945915809121066091270640911C
:108AC0009A052091280600912106E09098050E94C1
:108AD000141881E00E9427026DCF84E00E942A29A9
:108AE00083CF80E00E940E299091B306890F60E049
:108AF00040E00E948D1C29CF81E00E942A29DECE11
:108B0000991B79E004C0991F961708F0961B881FDF
:108B10007A95C9F780950895AA1BBB1B51E107C040
:108B2000AA1FBB1FA617B70710F0A61BB70B881FFD
:108B3000991F5A95A9F780959095BC01CD0108958C
:108B400097FB092E07260AD077FD04D0E5DF06D073
:108B500000201AF4709561957F4F0895F6F790956F
:108B600081959F4F0895A1E21A2EAA1BBB1BFD0100
:108B70000DC0AA1FBB1FEE1FFF1FA217B307E407FC
:108B8000F50720F0A21BB30BE40BF50B661F771F54
:108B9000881F991F1A9469F7609570958095909534
:0E8BA0009B01AC01BD01CF010895F894FFCFF9
:108BAE0001000100010001000100010001000100AF
:108BBE000100010001000100010001C00080004021
:108BCE00007F206430480F04050607111210130EA3
:108BDE0004050607111210130409050A06070B11E6
:108BEE000C120D101325212326272422201D1E1BB7
:108BFE00191F1C1A1012180F110C130E0B140D0A3C
:108C0E0015160917040508030601070002032019AB
:108C1E001A180C0B0A090420191A180C0B0A09222F
:108C2E0021252320191A18241B1C0F0E0D04030ACC
:108C3E000C0B0908010200201B191C1A180F0C0E30
:108C4E000B0D0A0926271D1E1F10121113141516BF
:108C5E00170506076E306E783078000100070E0992
:108C6E001C1B1215383F363124232A2D70777E793E
:108C7E006C6B6265484F464154535A5DE0E7EEE92E
:108C8E00FCFBF2F5D8DFD6D1C4C3CACD90979E991E
:108C9E008C8B8285A8AFA6A1B4B3BABDC7C0C9CE0E
:108CAE00DBDCD5D2FFF8F1F6E3E4EDEAB7B0B9BEFE
:108CBE00ABACA5A28F88818693949D9A2720292EEE
:108CCE003B3C35321F18111603040D0A5750595EDE
:108CDE004B4C45426F68616673747D7A898E8780CE
:108CEE0095929B9CB1B6BFB8ADAAA3A4F9FEF7F0BE
:108CFE00E5E2EBECC1C6CFC8DDDAD3D4696E6760AE
:108D0E0075727B7C51565F584D4A4344191E17109D
:108D1E0005020B0C21262F283D3A33344E4940478D
:108D2E0052555C5B7671787F6A6D64633E3930377D
:108D3E0022252C2B0601080F1A1D1413AEA9A0A76D
:108D4E00B2B5BCBB9691989F8A8D8483DED9D0D75D
:108D5E00C2C5CCCBE6E1E8EFFAFDF4F30409050A4F
:108D6E0006070B110C120D1013000100010001007B
:108D7E0001000100010001000100010001000100DD
:108D8E00010001C000800040000606011718191AE4
:108D9E001B1C1D1E1F202122233F3F3F0B0C0D0EBF
:108DAE000F10111213141516173F3F3F23242526BB
:108DBE002728292A2B2C2D2E2F3F3F3F1718191A03
:0E8DCE001B1C1D1E1F202122233F3F3F1500AE
:00000001FF
